:1000000000400020E1590000215A0000235A00005E
:1000100000000000000000000000000000000000E0
:10002000000000000000000000000000255A000051
:100030000000000000000000275A0000295A0000BC
:100040002B5A00002B5A0000156200002B5A0000AA
:100050002B5A0000000000002B5A00002B5A000011
:100060002B5A0000595C00002B5A00002B5A00004C
:100070002B5A00002B5A00002B5A00002B5A00006C
:100080002B5A0000B96200002B5A00002B5A0000C6
:100090002B5A00002B5A00002B5A00002B5A00004C
:1000A0002B5A00002B5A0000000000000000000046
:1000B0000000000000000000000000000000000040
:1000C000054B0648033310B51B1A062B03D9044B06
:1000D000002B00D0984710BD3402002034020020CD
:1000E000000000000648074910B5091A8910CB0F17
:1000F0005918491003D0044B002B00D0984710BD6D
:1001000034020020340200200000000010B5074C2B
:100110002378002B09D1FFF7D3FF054B002B02D02A
:10012000044800E000BF0123237010BD340200200A
:100130000000000070A50000094B10B5002B03D093
:100140000849094800E000BF08480368002B02D1B5
:10015000FFF7C8FF10BD064B002BF9D09847F7E713
:10016000000000003802002070A5000030020020CE
:1001700000000000164B002B00D1144B9D4640227E
:1001800092029A1A924600218B460F461348144A4F
:10019000121A07F09AFF0F4B002B00D098470E4B16
:1001A000002B00D098470020002104000D000D48CE
:1001B000002802D00C4800E000BF07F043FF2000F9
:1001C000290006F03FF807F017FFC04600000800BE
:1001D0000040002000000000000000003402002069
:1001E0005424002000000000000000000123034010
:1001F0000200181E04D1042A03D91068000900E087
:100200000020704710B50400FFF7F0FF0300002046
:1002100083420BD0013B9B00181DE2181279002A83
:1002200003D001338342F8D100E0180010BD012251
:10023000016810B5114201D0002903DA102000F046
:10024000AFF903E04910062001F0E8FE10BD016897
:1002500010B5CB0701D5002903DA102000F0A0F972
:1002600006E04910033189100022052001F0D6FE76
:1002700010BD70B50568AB0728D1042D26D90F2312
:100280002A6846681340062B09D12800FFF7AEFF05
:10029000012383421DDC9A00AE500133F9E7052BA0
:1002A00014D1F30703D4132000F07AF912E076108A
:1002B000FF2EF8D82800FFF799FF2C1D230080009F
:1002C0002018984205D91E700133FAE70B2000F080
:1002D00067F9002070BD70B50468E30701D41120F0
:1002E0002DE04568AB0729D1042D27D90F262B68AF
:1002F00064101E40062E0BD1002C04DD2800FFF7F1
:1003000075FF844201DD122019E0A400605918E055
:10031000331F012B12D82800FFF768FF8000042E3E
:1003200002D12800FFF76EFF002CECDDA042EADBD3
:1003300001232C19E0784000184302E00B2000F064
:100340002FF970BDF8B5012304681C4201D11120BA
:100350002FE00325466835402AD1042E28D90F23E3
:100360003268641087681340062B0BD1002C04DD23
:100370003000FFF73BFF844201DD122019E0A400AA
:10038000A75113E0052B13D1002CF6DD3000FFF749
:100390002DFF80008442F0DC01231F4201D1132095
:1003A00007E07F10FF2FFAD83419E770280002E029
:1003B0000B2000F0F5F8F8BD006810B5830717D1E1
:1003C000042815D90F2302681340062B02D1FFF72A
:1003D0000DFF0BE0052B05D1FFF708FFC00001233F
:1003E000184308E0042B03D1FFF70CFF4000F6E7A9
:1003F0000B2000F0D5F810BD10B5032400680440B0
:1004000006D1042804D90F2302681340042B01D01D
:100410000E2011E001F03EFE0378233B5942594182
:1004200010224018210008F029FB80239B05C218E8
:10043000054B9A4203D9142000F0B2F802E00123E0
:100440004000184310BDC046FFFFFF3F012303409B
:100450000200181E01D0501002E00D22014B1A704C
:100460007047C04650020020012303400200181EBE
:1004700004D1042A03D91068000900E00020704765
:1004800070B50D000400FFF7EFFF86002800FFF7AE
:10049000EBFF830000209E420ED1231D9E190435E0
:1004A0001A009E4207D929781278013301358A4211
:1004B000F6D0002000E0012070BD0000F0B585B04E
:1004C0000393019002912D4E2D4B002A02D002225F
:1004D0003270013A00251A601B68F554019B9D4259
:1004E0004ADA029AAB00D058254B1C68C8239B00FF
:1004F00037191C1B0123184202D04310214A1FE068
:10050000214A002802D0042805D1204A21003800C1
:1005100008F0A2F918E0042810D90F23026813404C
:10052000042B04D101F0B6FD194A030008E0062BA4
:1005300005D1FFF799FF174A030001E00123164A8E
:100540002100380008F088F9300008F0EBF9039B2F
:100550000B4A002B01D110600CE0019B013B9D4236
:10056000F9DA0E4B9842F6DC431C13602022325419
:100570000022F2540135B1E705B0F0BD5C02002065
:1005800058020020499800001C98000022980000A2
:10059000599B000027980000389800001F030000B6
:1005A000014B1870002070475002002070B502F017
:1005B00003FF094C0100251D1F22280008F0B9F98E
:1005C000280008F0AFF90423043080080001184324
:1005D0002060200070BDC0467C050020C368F0B5D7
:1005E0009D00836889B05D19030018330693036981
:1005F00003909F00069BDF1943699E000193069BB1
:100600009E19D24B1B78002B0FD17F222B68D0492B
:100610001C1213409B005B5801960435029235E092
:10062000CA4B1B78002B29D0019E039BC74C9B68AB
:1006300021780193EA1A039B92109B7812021A43C5
:10064000039B587802F044FC0023039A2370137034
:1006500001960497039B069A9B68ED1A0293039BED
:10066000AD10DD60049B9F1A039BBF101F61019BAF
:100670009B1A039A9B10536101F01EFC2B68029A8F
:100680001C121340B24A9B009B5804359F46039BA3
:10069000587802F015FC0023039A1370D9E7069BE3
:1006A0003A1DD11AA94BDB2903DD1A22019E1A70CB
:1006B000BBE71B783C60002B02D0019E1700B4E71B
:1006C0002B6802991C120B40A1499B005B58170034
:1006D0000435DBE7069B3A1DD11A9C4BDB2903DD71
:1006E0001A22019E1A70A0E728681B78291D38601D
:1006F000002B03D0019E17000D0096E76B6802994E
:100700001C120B4092499B005B5817000835BDE74F
:10071000069B3A1DD11A8D4BDB2903DD1A22019E5F
:100720001A7082E7A4001B782C193C60002B02D0C1
:10073000019E170079E72B6802991C120B4084492F
:100740009B005B5817000435A0E7069B3A1DD11AA1
:100750007E4BDB2903DD1A22019E1A7065E77D4876
:10076000A40021581B783960002B02D0019E17008D
:100770005BE72B6802991C120B4075499B005B5884
:100780001700043582E7043F724B3A68A400E25038
:100790006E4B1B78002B01D0019E46E72B68029A16
:1007A0001C1213406A4A9B009B5804356EE7694B44
:1007B000A600F058FFF74AFE043F04003868FFF730
:1007C00045FE24180120634B64000443F4505F4B42
:1007D0001B78002B01D0019E27E72B68029A1C1280
:1007E00013405B4A9B009B5804354FE7069B3A1D1C
:1007F000D11A564BDB2903DD1A22019E1A7014E729
:100800000198069C0121A04202D901000C39096817
:100810001B783960002B02D0019E170005E72B687A
:1008200002991C120B404A499B005B581700043583
:100830002CE7069B3A1DD11A444BDB2903DD1A2213
:10084000019E1A70F1E60199069881420AD90B00BF
:100850000C3B1B6840495B106418E41A019BA40020
:10086000E35802E01821197000233B60374B1B78D6
:10087000002B02D0019E1700D7E62B6802991C12AC
:100880000B4033499B005B5817000435FEE6019B83
:10089000069A93420BD90C3B19682F4B043FE3187F
:1008A0004910591A3A68019B8900CA5002E018227F
:1008B000264B1A70254B1B78002B01D0019EB4E605
:1008C0002B68029A1C121340214A9B009B58043546
:1008D000DCE6019B069A93421CD9019E1E4B0C3EFE
:1008E000E4183368019A5B10E31A9B009858FFF7ED
:1008F000ADFD043F04903868FFF7A8FD3168049B04
:100900004910611A012418184000019B89002043F6
:10091000C85002E018220D4B1A700C4B1B78002BAC
:1009200001D0019E81E62B68029A1C121340084AEE
:100930009B009B580435A9E6069B3A1DD11A034B30
:10094000DB290BDD1A22019E1A706EE65002002090
:100950001C960000BC220020FDFFFF3F0199A4006F
:1009600061581B783960002B02D0019E17005CE6AD
:100970002B6802991C120B40D0499B005B58170052
:10098000043583E6043F019B3A68A400E250CC4B57
:100990001B78002B01D0019E47E62B68029A1C129F
:1009A0001340C64A9B009B5804356FE6019BA40088
:1009B0001C192368043F38685E10FFF747FD36189E
:1009C0000120BF4B76001B7806432660002B01D028
:1009D000019E2AE62B68029A1C121340B74A9B001C
:1009E0009B58043552E6069BA4003F1BB44CBB4207
:1009F0000DD82378002B01D0019E16E62B68029AB1
:100A00001C121340AD4A9B009B5804353EE6AD488E
:100A100001F0B6FA2378002B01D0019E05E62B6881
:100A2000029A1C121340A54A9B009B5804352DE6E0
:100A3000A300ED18002C00DA0BE6A14B1B78002B6D
:100A400001D0019EF1E52B68029A1C1213409B4ACB
:100A50009B009B58043519E63B1F04931B680793C2
:100A6000042B04D1A300ED18002C00DAF2E5944B1E
:100A70001B78002B02D0019E049FD6E52B68029ABA
:100A80001C1213408D4A9B009B58049F0435FDE5C2
:100A90003B1F04931B68042B06D0A200AD18002C4A
:100AA00002DA002B00D1D5E5854B1B78002B02D054
:100AB000019E049FB9E52B68029A1C1213407F4ADD
:100AC0009B009B58049F0435E0E53A1F13685B10B8
:100AD000013B002B07DD01215B00A4000B430497C1
:100AE0002D191360B6E5764B17001B78002B01D04B
:100AF000019E9AE52B68029A1C1213406F4A9B00D4
:100B00009B580435C2E53A00069B0C32D31ADB2B06
:100B100004DD1A226A4B019E1A7086E5FF236100EC
:100B20005B000B4001210B433B60039B06989B68D5
:100B300024120493ED1A039BAD109B782D021D43E4
:100B4000019B8D401B1A9B108B400B43BB60039B8A
:100B50000D437D609C70E4B25B4BE4000399E35865
:100B600016008B6056490978002903D008331D0010
:100B700017005AE51D0002999B680C351C120B40AA
:100B80004E499B005B58019217007FE53B1F1E6892
:100B9000069A019B93422AD104970A20F30716D4A0
:100BA000B3070DD1042E0BD90F2332681340042B49
:100BB00006D1300001F06EFA07F0B4FE063006E010
:100BC0000720042E03D0002E01D080208000643046
:100BD00001F026FF002801D1043D3BE5039B3100D5
:100BE000587802F087F90023039A137032E5019BCD
:100BF000019A0C3B1B6803995B109B005B421F0032
:100C0000D3180C3B1E601300083B1B68083FD71924
:100C10005A108A70D2B22C49D2005B0055589B0AF8
:100C2000039A9B009560ED18019B043B1E68069B90
:100C30007610B6009E19224B1B78002B00D0F4E4EE
:100C40002B68029A1C1213401C4A9B009B58019669
:100C500004351BE53B1F1868FFF7F8FBA4000600EE
:100C60003F1B1E2834DC00280EDC154B1B78002BA4
:100C700001D0019ED9E42B68029A1C1213400F4A3E
:100C80009B009B58043501E502F07CFB033E3618BF
:100C900002F078FB0D4B801B9842F9D8084B1B786B
:100CA000002B01D0019EC0E42B68029A1C12134055
:100CB000024A9B009B580435E8E4C0461C9600009D
:100CC000500200204C980000C41A00209F860100AA
:100CD0000123039A137002F055FB039B0A3886190F
:100CE0005E60B6E43B1F1868FFF7B0FBA4000490F9
:100CF0003F1B00280EDCCF4B1B78002B01D0019E40
:100D000093E42B68029A1C121340CB4A9B009B5819
:100D10000435BBE4C94B049A019E9A4203DD1D22AF
:100D2000C44B1A7081E40123039A137002F02AFB6A
:100D3000FA23049A9B005343039A0A3B1B185360FF
:100D400087E4A300FF1A002320001A003900FFF7F0
:100D5000B5FBBB4EBB4C3168200002F017F8316880
:100D6000200002F0CEF8B34B1B78002B01D0019E7F
:100D70005BE42B68029A1C121340AF4A9B009B58FD
:100D8000043583E4AB4BA4001B783F1B002B01D040
:100D9000019E4AE42B68029A1C121340A64A9B004B
:100DA0009B58043572E401F081FE01F085F83B1F89
:100DB0001868002823D1083B1868C30701D54010E4
:100DC00016E083070FD104280DD90F2302681340C2
:100DD000062B02D1FFF748FB0AE0052B03D1FFF7F2
:100DE00043FB800004E01922924B019E1A701CE420
:100DF0003A0001214300083A0B43136001E0401020
:100E00000138002832DD012243001343391F0B60F3
:100E10003B00083B1B681341181A3B000C3B1B6846
:100E2000134203D08018A400904015E0990717D111
:100E3000042B15D90F211E683140062906D1013037
:100E40008000C358019AA400A35010E0052907D1DF
:100E500018180079A4004000019B1043E05006E000
:100E60001922744B019E1A70FFF7DFFB0435714B9A
:100E70001B78002B02D0019EFFF7D7FB2B68029A4C
:100E80001C1213406C4A9B009B580435FFF7FEFB75
:100E9000A300069AFB189B1ADB2B01DC012205E05C
:100EA0001A22644B019E1A70FFF7BFFB631E002CD1
:100EB00003DD3A601C000437F8E75E4B1B78002B1B
:100EC00002D0019EFFF7B1FB2B68029A1C1213405F
:100ED000594A9B009B580435FFF7D8FBA3009C465A
:100EE000F81A002C04DC1C22524B00261A7015E064
:100EF000002103685B1001268A008258164003D146
:100F00000D224C4B1A7009E05210934200DD130081
:100F100001318C42EFDC01265B001E436346FF1A61
:100F2000444B06601B780437002B02D0019EFFF76C
:100F30007CFB2B68029A1C1213403F4A9B009B5873
:100F40000435FFF7A3FBA3009C46F81A002C04DC31
:100F50001C22384B00261A7015E0002103685B1034
:100F600001268A008258164003D10D22314B1A7097
:100F700009E05210934200DA130001318C42EFDC99
:100F800001265B001E436346FF1A2A4B06601B784E
:100F90000437002B02D0019EFFF747FB2B68029A13
:100FA0001C121340244A9B009B580435FFF76EFB2C
:100FB0003B00083B1868FFF749FA3B1F049018688C
:100FC000FFF744FA049AA600BC1B0023824200DA11
:100FD00004332360174BBF1B1B780437002B02D050
:100FE000019EFFF722FB2B68029A1C121340124A43
:100FF0009B009B580435FFF749FBA300FE1A04939E
:101000003B00083B1868FFF721FA3B1F04001868F3
:10101000FFF71CFAE20FC317A04253419B00336055
:10102000049BFF1A034B04371B78002B0CD0019E46
:10103000FFF7FBFA500200201C96000080EE3600FD
:10104000580200205C0200202B68029A1C121340F8
:10105000DB4A9B009B580435FFF718FB3B00083B1D
:1010600018683B1F1968A300884202D1FB1A0422AA
:1010700022E004281ED90122104201D0114219D1C8
:101080000326304215D10F2302681A40042A10D1DA
:1010900031420ED104290CD90A681340042B08D11F
:1010A000FFF7EEF9431E9841A600BE1B800030609A
:1010B00003E0A3000022FB1A1A60C24BA4001B78B5
:1010C0003F1B0437002B02D0019EFFF7AEFA2B68BE
:1010D000029A1C121340BA4A9B009B580435FFF732
:1010E000D5FA3B00083B18683B1F1968A3008842EB
:1010F00002D1FB1A002226E0042822D90122104244
:1011000004D0114202D0FB1A03321CE00326304205
:1011100016D10F2302681A40042A11D131420FD18F
:1011200004290DD90A681340042B09D1FFF7A8F947
:10113000030058425841A600BE1B8000306003E007
:10114000A3000422FB1A1A609E4BA4001B783F1BCD
:101150000437002B02D0019EFFF767FA2B68029A32
:101160001C121340964A9B009B580435FFF78EFAD9
:10117000A300FE1A04933B00083B1868FFF766F9CA
:101180003B1F04001868FFF761F9E217C30F8442A0
:1011900053419B003360049BFF1A8A4B04371B7832
:1011A000002B02D0019EFFF740FA2B68029A1C1216
:1011B0001340834A9B009B580435FFF767FA3B00B6
:1011C000083B1868FFF742F93B1F04901868FFF7C7
:1011D0003DF9049AA600BC1B0023824200DD0433C3
:1011E0002360784BBF1B1B780437002B02D0019E75
:1011F000FFF71BFA2B68029A1C121340704A9B00DF
:101200009B580435FFF742FA3B1F1B68A400043BC0
:10121000591E8B413A1B17009B001360694B043722
:101220001B78002B02D0019EFFF7FFF92B68029A72
:101230001C121340624A9B009B580435FFF726FAA4
:10124000A300FC1A04933B00083B1868FFF7FEF864
:101250003B1F06001868FFF7F9F836180120049BB9
:101260007600FF1A574B06431B7826600437002B85
:1012700002D0019EFFF7D9F92B68029A1C12134085
:101280004F4A9B009B580435FFF700FAA300FE1A53
:1012900004933B00083B1868FFF7D8F83B1F040095
:1012A0001868FFF7D3F8241A0120049B6400FF1A82
:1012B000444B04431B7834600437002B02D0019E5A
:1012C000FFF7B3F92B68029A1C1213403C4A9B00AB
:1012D0009B580435FFF7DAF9A300FC1A04933B008E
:1012E000083B1868FFF7B2F83B1F06001868FFF7C5
:1012F000ADF846430120049B7600FF1A314B0643AC
:101300001B7826600437002B02D0019EFFF78DF971
:101310002B68029A1C121340294A9B009B580435E3
:10132000FFF7B4F93B00083B1868FFF78FF83B1F45
:1013300004901868FFF78AF80100049805F08AF80D
:101340000123A4003E1B3700400018431D4B3060B2
:101350001B780437002B02D0019EFFF766F92B683B
:10136000029A1C121340164A9B009B580435FFF743
:101370008DF93B00083B1868FFF768F83B1F0490A5
:101380001868FFF763F80100049805F049F9012394
:10139000A4003E1B3700490019430A4B31601B78FB
:1013A0000437002B02D0019EFFF73FF92B68029A09
:1013B0001C121340024A9B009B580435FFF766F944
:1013C0001C960000500200203B1F1868FFF73EF8F3
:1013D000C317C01858400123A4003E1B370040002B
:1013E0001843EA4B30601B780437002B02D0019E73
:1013F000FFF71BF92B68029A1C121340E44A9B006A
:101400009B580435FFF742F9A300FE1A0793306892
:10141000012C03D1FFF71AF8049008E0FFF716F843
:1014200004007068FFF712F80130031B0493049B5B
:10143000002B01DC0123049307F0C0F9049905F0A7
:10144000EFF80C190121079B6400FF1ACF4B0C43E6
:101450001B7834600437002B02D0019EFFF7E5F8BB
:101460002B68029A1C121340C94A9B009B580435F2
:10147000FFF70CF9A4003E1B3000FEF7BDFF37005C
:10148000C24B30601B780437002B02D0019EFFF75F
:10149000CCF82B68029A1C121340BD4A9B009B5843
:1014A0000435FFF7F3F8A300FE1A04933B00083B52
:1014B0001868FEF7CBFF3B1F04001868FEF7C6FF55
:1014C00004400120049B6400FF1AB04B04431B78C6
:1014D00034600437002B02D0019EFFF7A6F82B687A
:1014E000029A1C121340AA4A9B009B580435FFF72E
:1014F000CDF8A300FC1A04933B00083B1868FEF7E4
:10150000A5FF3B1F06001868FEF7A0FF0643012059
:10151000049B7600FF1A9D4B06431B782660043718
:10152000002B02D0019EFFF780F82B68029A1C1254
:101530001340974A9B009B580435FFF7A7F8A30078
:10154000FC1A04933B00083B1868FEF77FFF3B1F23
:1015500006001868FEF77AFF46400120049B7600DB
:10156000FF1A8A4B06431B7826600437002B02D0F3
:10157000019EFFF75AF82B68029A1C121340844A06
:101580009B009B580435FFF781F83B1F1868FEF756
:101590005DFFC0430123A4003E1B370040001843F9
:1015A0007A4B30601B780437002B02D0019EFFF786
:1015B0003CF82B68029A1C121340754A9B009B58FA
:1015C0000435FFF763F8A300FE1A04933B00083BC1
:1015D0001868FEF73BFF3B1F04001868FEF736FF54
:1015E0008440012364001C43049B3460FF1A674B52
:1015F00004371B78002B02D0019EFFF716F82B68EA
:10160000029A1C121340624A9B009B580435FFF754
:101610003DF8A300FE1A04933B00083B1868FEF750
:1016200015FF3B1F04001868FEF710FF044101235B
:1016300064001C43049B3460FF1A544B04371B782E
:10164000002B02D0019EFEF7F0FF2B68029A1C12BD
:1016500013404F4A9B009B580435FFF717F83B0097
:101660000C3B1868FEF7F2FE3B00083B06001868CA
:10167000FEF7ECFEF1170200C317300005F022F868
:101680003B1F049005911868FEF7E0FE02000498E5
:10169000059904F0CBFF0123A4003E1B3700400056
:1016A00018433A4B30601B780437002B02D0019E60
:1016B000FEF7BBFF2B68029A1C121340344A9B00B2
:1016C0009B580435FEF7E2FFA4003E1B3000FEF7F6
:1016D000AEFD37002D4B30601B780437002B02D055
:1016E000019EFEF7A2FF2B68029A1C121340284AA3
:1016F0009B009B580435FEF7C9FFA4003E1B300039
:10170000FEF7A5FD3700214B30601B780437002B16
:1017100002D0019EFEF789FF2B68029A1C1213402B
:101720001B4A9B009B580435FEF7B0FFA4003F1BEB
:101730003800FEF79EFD154B1B78002B02D0019E52
:10174000FEF773FF2B68029A1C121340104A9B008D
:101750009B580435FEF79AFFA4003E1B3000FEF7AD
:10176000BAFD3700094B30601B780437002B02D0DC
:10177000019EFEF75AFF2B68029A1C121340044A7E
:101780009B009B580435FEF781FFC04650020020A5
:101790001C960000A4003F1B3800FEF7D3FDE64B6B
:1017A0001B78002B02D0019EFEF73FFF2B68029AA8
:1017B0001C121340E14A9B009B580435FEF766FF5C
:1017C000A4003E1B3000FEF7F7FD3700DA4B306017
:1017D0001B780437002B02D0019EFEF726FF2B68F2
:1017E000029A1C121340D54A9B009B580435FEF701
:1017F0004DFF069A3B1D0493CF4C9B1ADB2B04DD57
:101800001A23019E2370FEF710FF01F0C5FD01238E
:101810004000184323783860002B03D0019E049FBA
:10182000FEF703FF2B68029A1C121340C34A9B0069
:101830009B58049F0435FEF729FF069A3B1D04932D
:10184000BD4C9B1ADB2B04DD1A23019E2370FEF78F
:10185000ECFE01F097FDBA4B4000184001231843FD
:1018600023783860002B03D0019E049FFEF7DDFE35
:101870002B68029A1C121340B04A9B009B58049F8D
:101880000435FEF703FFA300FB1A04930123200095
:101890001A000499FEF712FEAA4C2068643001F089
:1018A000BFF8002816D0039B21685A78A64801F09B
:1018B00036FB15E0A300FB1A04932000012300224D
:1018C0000499FEF7FBFD9F4C2068643001F0A8F8F6
:1018D000002802D1043DFEF7BCFE9B4801F0BAF996
:1018E0000123039A137001F04DFDC8222368D20032
:1018F000063353431818039B5860FEF7ABFEA40051
:101900003E1BFEF753FE37008B4B30601B780437CD
:10191000002B02D0019EFEF788FE2B68029A1C1253
:101920001340864A9B009B580435FEF7AFFEA40087
:101930003E1B300001F064FD37007F4B30601B78A8
:101940000437002B02D0019EFEF76FFE2B68029A2F
:101950001C121340794A9B009B580435FEF796FEF3
:10196000A4003E1B300001F04DFD3700724B30608B
:101970001B780437002B02D0019EFEF756FE2B6821
:10198000029A1C1213406D4A9B009B580435FEF7C7
:101990007DFEA4003E1B300001F036FD3700664B93
:1019A00030601B780437002B02D0019EFEF73DFE0D
:1019B0002B68029A1C121340604A9B009B58043506
:1019C000FEF764FEA4003F1B380001F03BFD5A4BBC
:1019D0001B78002B02D0019EFEF727FE2B68029A8F
:1019E0001C121340554A9B009B580435FEF74EFECF
:1019F000A300FE1A31002000049301F045FD049B72
:101A00003060FF1A4C4B04371B78002B02D0019E2C
:101A1000FEF70BFE2B68029A1C121340474A9B00EC
:101A20009B580435FEF732FEA4003F1B380001F03E
:101A300065FD414B1B78002B02D0019EFEF7F5FDA2
:101A40002B68029A1C1213403C4A9B009B58043599
:101A5000FEF71CFE0121200001F038FD364B1B78FB
:101A6000002B02D0019EFEF7E0FD2B68029A1C12AB
:101A70001340324A9B009B580435FEF707FE0021B5
:101A8000200001F023FD2C4B1B78002B02D0019E7F
:101A9000FEF7CBFD2B68029A1C121340274A9B00CD
:101AA0009B580435FEF7F2FDA4003E1B300001F008
:101AB00043FD3700204B30601B780437002B02D0E9
:101AC000019EFEF7B2FD2B68029A1C1213401B4ABE
:101AD0009B009B580435FEF7D9FDA4003E1B300047
:101AE00001F03EFD3700144B30601B780437002BAB
:101AF00002D0019EFEF799FD2B68029A1C1213403A
:101B00000E4A9B009B580435FEF7C0FDA4003F1B06
:101B1000380001F0FFFC084B1B78002B02D0019E1F
:101B2000FEF783FD2B68029A1C121340034A9B00A8
:101B30009B580435FEF7AAFD500200201C960000B9
:101B4000FEFFFF7F580200205C020020A4003F1B24
:101B5000380002F005FAD94B1B78002B02D0019E09
:101B6000FEF763FD2B68029A1C121340D44A9B00B7
:101B70009B580435FEF78AFDA4003E1B300002F09E
:101B800099FA3700CD4B30601B780437002B02D018
:101B9000019EFEF74AFD2B68029A1C121340C84AA8
:101BA0009B009B580435FEF771FDA4003F1B3800D5
:101BB00002F0A6F9C14B1B78002B02D0019EFEF764
:101BC00034FD2B68029A1C121340BD4A9B009B589F
:101BD0000435FEF75BFDA4003E1B300002F0A6F9C1
:101BE0003700B64B30601B780437002B02D0019EC3
:101BF000FEF71BFD2B68029A1C121340B04A9B0093
:101C00009B580435FEF742FDA4003F1B380001F04D
:101C10009DFFAA4B1B78002B02D0019EFEF705FD0D
:101C20002B68029A1C121340A54A9B009B5804354E
:101C3000FEF72CFDA4003F1B380001F09DFF9F4BD9
:101C40001B78002B02D0019EFEF7EFFC2B68029A56
:101C50001C1213409A4A9B009B580435FEF716FD50
:101C6000A4003F1B380001F097FF944B1B78002B1A
:101C700002D0019EFEF7D9FC2B68029A1C12134079
:101C80008F4A9B009B580435FEF700FDA4003F1BC4
:101C9000380001F0A9FF894B1B78002B02D0019E70
:101CA000FEF7C3FC2B68029A1C121340844A9B0067
:101CB0009B580435FEF7EAFCA300FE1A3100200011
:101CC000049302F038FA049B3060FF1A7B4B043710
:101CD0001B78002B02D0019EFEF7A7FC2B68029A0E
:101CE0001C121340764A9B009B580435FEF7CEFC2D
:101CF000A300FE1A31002000049302F034FA049B82
:101D00003060FF1A6D4B04371B78002B02D0019E08
:101D1000FEF78BFC2B68029A1C121340684A9B004A
:101D20009B580435FEF7B2FCA300FE1A31002000D8
:101D3000049302F0DAF9049B3060FF1A5F4B04371A
:101D40001B78002B02D0019EFEF76FFC2B68029AD5
:101D50001C1213405A4A9B009B580435FEF796FC10
:101D6000A300FE1A31002000049302F0D7F9049B6F
:101D70003060FF1A514B04371B78002B02D0019EB4
:101D8000FEF753FC2B68029A1C1213404C4A9B002E
:101D90009B580435FEF77AFCA4003F1B380001F085
:101DA0004BFF464B1B78002B02D0019EFEF73DFCFB
:101DB0002B68029A1C121340414A9B009B58043521
:101DC000FEF764FCA300FF1A3900200001F0EAFFCF
:101DD0003A4B1B78002B02D0019EFEF726FC2B68A5
:101DE000029A1C121340364A9B009B580435FEF79A
:101DF0004DFCA4003E1B300001F0A0FF37002F4B2C
:101E000030601B780437002B02D0019EFEF70DFCDA
:101E10002B68029A1C121340294A9B009B580435D8
:101E2000FEF734FCA300FF1A3900200001F064FF24
:101E3000224B1B78002B02D0019EFEF7F6FB2B688D
:101E4000029A1C1213401E4A9B009B580435FEF751
:101E50001DFCA300FF1A3900200000F063FD174BA2
:101E60001B78002B02D0019EFEF7DFFB2B68029A45
:101E70001C121340124A9B009B580435FEF706FCC7
:101E8000A300FE1A31002000049300F04BFD049BD8
:101E90003060FF1A094B04371B78002B02D0019EDB
:101EA000FEF7C3FB2B68029A1C121340044A9B00E6
:101EB0009B580435FEF7EAFB09B0F0BD5002002044
:101EC0001C9600000023F7B55A1E0192002B07DA7A
:101ED00001F0E8FC00F094FF01F046F86423019360
:101EE00000263000194B19688E4201DB019BEBE79D
:101EF000174B1A680132914200DC0022F0241A606C
:101F00001D68144F6C43E35D002B1DD0E419022BB8
:101F100016D0012B0ED1002801D101F033FAF022A6
:101F20006A430C4B0C499B185B68C31A8B4201D85F
:101F30000223BB54F0235D43064BEB5C022B03D121
:101F40002000FEF74BFBD1E70136CBE7540200201F
:101F500000000020641100209F860100054B012134
:101F60001A68054B1A600023044AD1500433642BCD
:101F7000FBD17047A8050020A0050020BC2200204E
:101F800000B59BB00200054901A806F097FC01A826
:101F900000F07CFE00F0E8FFFCE7C0465C98000023
:101FA00037B5174D04002868002801D006F07AF8EC
:101FB000A400200006F06CF82860002801D1114828
:101FC00009E001AB984208D20F4B02196B44019310
:101FD000934202D20D48FFF7D3FF042802D80830FD
:101FE0002860083C2B680A4A1C191360094B012120
:101FF0001C600023084AD1500433642BFBD137BD49
:10200000A80500206D9800001CFCFFFF9D980000B3
:10201000A0050020A4050020BC22002070B50D4DB5
:102020000D4E2B684C1CA40036681C19B44203D911
:102030000A20FEF7B5FA0BE02C601D00AC4201D976
:1020400004C5FBE70F22090110400843186018007F
:1020500070BDC046A0050020A40500200322CB1CB3
:1020600070B50C00D9171140C9180500891000225D
:102070000420FFF7D3FF0023A34204DAE95CC2186F
:1020800011710133F8E7E1430023C91721404118DA
:102090000B7170BD10B5830706D1042804D90F2336
:1020A00004C81340042B03D00E20FEF779FA014830
:1020B00010BDC046AD99000070B501240B680D003D
:1020C0001C4001D05C1002E00D20FEF769FA2000F0
:1020D00004F038FC264904F021FB05F0FBFE02F079
:1020E0000FFB0022234B05F0AFF80023002204F081
:1020F000DFFA01242B681C40002819D0002C01D0E5
:102100005C1002E00D20FEF74BFA200004F01AFCF0
:10211000174904F003FB05F0DDFE02F0F1FA00229E
:10212000144B05F091F80022134B04F053FC18E017
:10213000002C01D05C1002E00D20FEF731FA2000E7
:1021400004F000FC0A4904F0E9FA05F0C3FE02F0CD
:10215000D7FA0022074B05F077F80022064B05F06E
:10216000EDFA05F03FFE01234000184370BDC04664
:10217000D30237390000D0400000E03F10B5034AD9
:102180000121034800F0BAFB10BDC0460400002046
:102190000899000030B502248025094B094AED005A
:1021A0009C505C59002CFCD0A124E400884204D24D
:1021B0008025ED0018514019F8E70021995030BDF5
:1021C00000E001400405000010B5002804D1E02023
:1021D0009C210002890203E09C2080218002C90228
:1021E000FFF7D8FF10BD002802D09C239B0201E01E
:1021F000E0231B021B6800201A0E532A01D11B0288
:10220000180A704730B501248025064A064BED00B8
:10221000D4505459002CFCD001600021014AD15007
:1022200030BDC04600E001400405000010B50028A4
:1022300002D09C20800201E0E0200002A6230902D7
:10224000DB05090A1943FFF7DDFF10BDF0B50124D6
:10225000802503000F4F08000F49ED007C507C598A
:10226000002CFCD09C46002810DD5478167893781A
:10227000240234431B0423431C00D37801381B067B
:102280002343644608C40432A446ECE700237B5091
:10229000F0BDC04600E001400405000070B5050037
:1022A0004B680A009C1C2100FFF7D0FFA0002818F3
:1022B00070BD0000154B1B68002B04D080219C23AF
:1022C000C9029B0203E09C21E02389021B02002833
:1022D00007D1191D5B6802001B0E522B14D10A0096
:1022E00012E0002281420FD903681B0E522B0BD142
:1022F000436802339B00C318994205D91A68110E2E
:102300000022522900D11A0010007047AC070020AB
:102310008022F0B5520085B00021624805F0D5FE5C
:10232000802200215200604805F0CFFE5F4B1B6801
:102330001A00029353425A4110000392FFF744FFE0
:10234000029B002B01D15A4C00E05A4C0020FFF7B1
:10235000B1FFFF270500002D00D194E02B681A1271
:102360001B143A403B4001921A000A3A092A43D80A
:102370004C4B019A995C002900D07FE010224E4816
:1023800005F0A3FE2E00336801991A123A409142DB
:1023900017D11A143A400B2A06D0132A0CD00A2A55
:1023A0000FD1454B1E600CE03B40022B09DC424A3A
:1023B0009B00D3185E6004E0102200213E4805F027
:1023C00084FE3000FFF776FF061EDCD13A4B196819
:1023D00000290FD02000FFF761FF0400374E31685D
:1023E000002903D02000FFF759FF0400344B0436C6
:1023F000B342F4D12B4B3EE0143B092B3ED82A4B81
:10240000019A995C002939D108222E4805F05DFE19
:102410002E0033681A143A40152A0BD01D2A11D009
:10242000142A14D1019A1B123B409A420FD1254B1A
:102430001E600CE0019A1B123B409A4207D1214BCF
:102440005E6004E0082200211E4805F03EFE3000D8
:10245000FFF730FF061EDCD11A4E3168002909D083
:102460002000FFF71BFF71680400002902D0FFF76E
:1024700015FF04000C4B0121019A99542800FFF725
:1024800019FF050067E70298FFF7ADFE411C0398AE
:10249000FFF7CCFE054B039A1A600B4B1C6005B08E
:1024A000F0BDC046AC060020AC050020AC07002003
:1024B0000470020004E000002023002024230020F8
:1024C0003023002030230020B007002070B500200A
:1024D000FFF789FE04000120FFF785FE844200DA41
:1024E00004000A4B1E687542754128001D60FFF705
:1024F0006BFE002E01D0064B00E0064B064A28007A
:10250000611C1360FFF792FE70BDC046AC0700204F
:1025100004E0000004700200B0070020F8B50020BD
:10252000FFF761FE07000120FFF75DFE3E00224D30
:102530000643224C0CD18021E020C9020002FFF7A3
:1025400029FE01213000FFF771FE2E601C4B2FE0A9
:10255000874208DD00239C212B60194B89022360F0
:102560002368002011E0012380212B60154BC90254
:102570002360F5E71A68551C18D0120E522A07D1AD
:1025800001205A68023292009B188B42F2D311E06C
:10259000002800D023600C4C0C49200006F0BAF94A
:1025A000200000F001FFFFF791FF04E0002802D0B7
:1025B000236000E02160F8BDAC070020B0070020D8
:1025C00004E0000004700200742300201E99000043
:1025D000F0B585B0039203220333DC1714402A4E72
:1025E000E3189C10336801900291002B02D08022E6
:1025F000D20201E09C229202244FA51C3B68AD0050
:102600005B199A4217D2FFF783FE3368002B02D082
:102610008022D20201E09C2292023B685B199A421E
:1026200009D21B4C1B49200006F074F9200000F071
:10263000BBFE002026E0029B3E681B06190C6B4681
:102640001A7BA423DB051343019A0B431104FF22D9
:102650001204114019433000FFF7D4FD3300301D40
:102660000833210001933B60FFF7CCFD002C04D020
:102670000A9A21000198FFF7E9FD3000019B083D0F
:102680005D193D6005B0F0BDAC070020B00700202B
:10269000742300204799000070B59AB0FFF73EFF01
:1026A000FF221F4CD2000021200005F00EFD00206B
:1026B000FFF700FEFF25002600281AD003681A1431
:1026C0002A400A2A08D11A122A40FF2A0ED0D20024
:1026D000A1180B71A05009E0132A07D11B122B403F
:1026E000FF2B03D0DB00E2181671E650FFF7E2FD86
:1026F000E2E7FF210200C900235808305D1EAB410C
:10270000D2188842F8D1074901A806F0D7F801A8E5
:1027100000F0BCFA044800F0B9FA1AB070BDC04627
:10272000C41A00206E9900008699000000207047AE
:102730000120704700487047502300200048704730
:1027400033F8FFFF10B50449044806F0E3F82423EA
:102750000348036010BDC046419A00003C2300209E
:102760003823002000207047002070470020704769
:1027700000207047002070470020704700207047FD
:10278000002070470020704710B5034A0E2103480F
:1027900000F0B4F810BDC0460C000020469A0000BE
:1027A000044A05491368C85401339B059B0D136007
:1027B0007047C046B80B0020B4070020114A70B51E
:1027C0001368114C984211DA015D451CFA39012950
:1027D00006D8AB4206DD2118497801391F2901D9F5
:1027E0002800EFE70100251A461C02D100231360E0
:1027F00006E0665C6E5401318B42FADC181A1060F8
:1028000070BDC046BC0B0020C40B002010B500F00A
:10281000B9FD064B1A68904201D200221A601B686B
:10282000C01A034B83428041404210BDC00B0020C0
:10283000204E000010B5094C094A236812689342E3
:102840000BD0084AD05C00F0E1FE002805D02368D8
:1028500001339B059B0D2360EDE710BDC40F0020E5
:10286000B80B0020B407002010B50400064B074A3F
:102870001B6812689B1ADB439B059B0DA34202DA7F
:10288000FFF7D8FFF2E710BDB80B0020C40F0020FF
:10289000F7B506000191151E2FD05768B800441CEB
:1028A0000630FFF7E1FFFB20FFF77AFF1C20FFF760
:1028B00077FFF0B2FFF774FFE0B22412FFF770FF6A
:1028C000E0B2FFF76DFF6B461879FFF769FF00264E
:1028D000BE4212DAB300EB189C680136E0B2FFF793
:1028E0005FFF2012C0B2FFF75BFF2014C0B2FFF7FA
:1028F00057FF200EFFF754FFEAE7F7BD70B5074D0D
:102900002C68092C08DC0C236343054E01349851D4
:10291000F31859609A602C6070BDC046C80F002043
:10292000D8230020F0B589B004900E0001284BDDBB
:10293000284B08680293830709D1042807D90F237D
:1029400002681340042B02D1FFF7A4FB0290214B35
:1029500070680393830709D1042807D90F230268FD
:102960001340042B02D1FFF795FB039000271A4B6D
:102970001A4D1B680593059B9F4225DA2B1F029970
:10298000186805F0BDFF00281BD12B686C68069302
:102990000190019B069A934213DA206803990794E9
:1029A00005F0AEFF0834002807D131000498079BDA
:1029B00008315B680238984709E0019B01330193B5
:1029C000E7E701370C35D6E71B20FDF7E9FD09B035
:1029D000F0BDC046AD990000C80F0020DC230020E8
:1029E00010B501F053FA00F0D1FDFFF7C7FB00F07E
:1029F00041FEFFF7C9FE01F0A7FA01F023FC10BD6C
:102A0000962210B512010021034805F05EFB00225A
:102A1000024B1A6010BDC046641100205402002011
:102A2000064B074A1B6812689B1ADB439B059B0DEC
:102A30000122834200DC002210007047B80B002006
:102A4000C40F0020F8B505000C0016001F1E0ED1A3
:102A50000320FFF7E5FF002827D0FA20FFF7A0FEAC
:102A6000E8B2FFF79DFEE0B2FFF79AFE1DE0501DB1
:102A7000FFF7D6FF002818D0FB20FFF791FEE8B241
:102A8000FFF78EFEE0B2FFF78BFEF0B2FFF788FE95
:102A90003012C0B2FFF784FE3C00E31B9E4204DD0F
:102AA0002078FFF77DFE0134F7E7F8BD70B500240C
:102AB000F0250B4B1B689C420EDA2A006243094B3F
:102AC000D3181A78002A05D05978002311201A004B
:102AD000FFF7B8FF0134ECE7FFF792FF70BDC04687
:102AE00054020020641100200123F3B50400FFB05C
:102AF0000D0010001A420DD002AA1370431002A953
:102B0000537042121B0E40148A700B71C8700B0078
:102B1000052273E0032313401ED1042A1CD90F227F
:102B200001680A40042A17D1023302AA1370FFF782
:102B3000B1FA060005F0F6FEF823FF33984200DDF7
:102B400018000023834205DA01335A1EB25C02A941
:102B5000CA54F7E7421C50E0042801D0002809D1EC
:102B6000032302AA043813704342434153701300F5
:102B7000022243E0002B45D1042843D90F210268EB
:102B80001140052912D1043302A90B70F823120950
:102B9000FF3392009A4200DD1A00002393422BDAA1
:102BA0000133C118C97802AEF154F7E7062929D1DB
:102BB00001390E00120956430196F826019FFF368F
:102BC000B7421FDC02AE31700136934213DA01279F
:102BD000013399004158394201D0394100E00A4996
:102BE000012737700F127170B7700F14090EF7704C
:102BF00031710536E9E7019A013202AB2900200064
:102C0000FFF720FF7FB0F3BD19FCFFFF70B5F02385
:102C1000050000240D4A1800604380184178A9423D
:102C200003D001340A2CF6D10FE0F022002105F088
:102C30004CFA074A1368013BA34200D114600023F9
:102C400029001A001120FFF7FDFE70BD641100205D
:102C50005402002010B5B2B002236A46040013707B
:102C600005F060FEC72800DDC7200023834205DA97
:102C7000694601335A1EA25CCA54F7E7421C6B46F0
:102C8000FE211420FFF7DEFE32B010BD10B5B2B049
:102C900002236A460400137005F044FEC72800DDD5
:102CA000C7200023834205DA694601335A1EA25C1D
:102CB000CA54F7E7421C6B46FF211420FFF7C2FEFF
:102CC00032B010BDF7B5234B06001B68F02000930F
:102CD00000232149009A93420ADA02005A438A18D3
:102CE0005478B44202D11278002A31D10133F1E78D
:102CF0000024F0231A00624301920199164A5518E4
:102D00002F78002F06D001340A2CF3D11348FFF797
:102D1000BDFF1DE0F0223900280005F0D6F902239E
:102D20000D4A0199EB6053540D4AF1008A58009BFB
:102D30006E70AE70AA602F616F61A34202DC054B1A
:102D400001341C60002331001A001020FFF77AFEC6
:102D5000F7BDC0465402002064110020019B000012
:102D6000C41A002010B5FFF7A1FE0024064BE200B4
:102D7000D3181B79043B012B02D8E0B2FFF7A2FF66
:102D80000134FF2CF2D110BDC41A0020F7B50E009B
:102D900000247F250190194BE200D11809790629FA
:102DA00001D0032926D1985883682B401C2B21D1B0
:102DB000C3681A002A40042A1CD102692A40192A31
:102DC00018D11B0A01339B000C30C018FFF762F9C1
:102DD000070005F0A7FD0023B0420BD19E4206DD9F
:102DE000019AF95CD25C914204D10133F6E7E0B27A
:102DF000FFF768FF0134FF2CCDD1F7BDC41A0020C6
:102E000070B500F0BFFA184B1A68904201D2002248
:102E10001A601A681549821A8A4223D9186000205C
:102E200000F08AFB444244416042072404430020EE
:102E300000F096FB002810D0082600250C4BEA0075
:102E4000D3181B799C4201D0B34202D1E8B2FFF7FC
:102E500039FF0135FF2DF1D104E0631C02D00126BA
:102E60007642EAE770BDC046B40B00200F27000091
:102E7000C41A002037B500240500FFF717FE01A88B
:102E8000019400F047FB200000F076FE00F00AFD00
:102E900000F07AFB00F079FB00F046FF00F09EFAAC
:102EA0000548FFF7F3FEA54204D0FFF757F80348A3
:102EB000FFF7ECFE37BDC046169B00002E9B0000BE
:102EC000002310B501001A001120FFF7BBFD10BD53
:102ED00007B56B46197069465A7013128B7013143C
:102EE000120ECB700A716B46010005221320FFF70A
:102EF000A9FD07BD10B50A0001001220FFF7F4FD7F
:102F000010BD70B5050008000C003230FFF7ACFCB6
:102F10002B00220000211B20FFF794FD70BD10B58F
:102F20000C000300110014202200FFF78BFD10BDE0
:102F300070B506000020FFF7BDF90024FF2500282A
:102F400010D003681A142A40152A05D11B122B40F1
:102F5000B34204D1040002E01D2A00D10024FFF78F
:102F6000A9F9ECE7200070BDF0B580279DB0FFF710
:102F700061FCB94DB94C2868FF00391A201800F0DF
:102F80002BFB2B680600C3182B60002B00D1DBE164
:102F9000002E0DDD2868391A201800F01DFB2B6863
:102FA00006001B182B6000F0EDF9AD4B1860EFE741
:102FB0002378FA2B00D00CE12B68022B06DCFFF7FC
:102FC00025FC002800D1BFE10120B8E16078A57898
:102FD0000238182800D9FAE003F0A8F90D1E2226BD
:102FE0002932F93D676F7589DAEFF9F9F9F9F9F9DD
:102FF000F9F9F9F9F300FF2D00D1E8E02800FFF717
:1030000005FE00229749EB005A50CB181A7129008F
:103010000092130013204DE02800FFF753FED6E086
:103020002800FFF7F3FDD2E0FFF79CFECFE0FFF7AB
:103030003DFD0020FFF71EFF8B48FFF727FEC6E08F
:10304000182D00D9C3E0894BAA00D25829001520B9
:10305000FFF74AFDBBE000242000FFF769FF071ED1
:1030600003D10134192CF7D1B1E0083005F05AFC36
:1030700006000530FFF7F8FBFB20FFF791FB1D2052
:10308000FFF78EFBE0B2FFF78BFBF0B2FFF788FB98
:103090003012C0B2FFF784FB0025AE42E1DD7B19A0
:1030A000187AFFF77DFB0135F7E700211D200B00A3
:1030B0000A000091FFF78CFA89E0002229000092B3
:1030C00013002720F6E700F077F903AC684A642183
:1030D0000090684B200005F0BFFB02232000237006
:1030E00005F020FC23000200002116206DE00024E2
:1030F0005C4AE300D558002D46D06B689E00701DD9
:10310000FFF7B2FB2B00002532000833210001201D
:10311000FFF798FC0020FFF7CDF82E002F000028C5
:103120001DD0FF2103681A120A40A24214D11A14BA
:103130000A400B2A07D10B400DD0012B09D0022BDE
:1031400000D1FFE008E0132A06D100252E002F0051
:1031500002E0060000E00700FFF7ACF8DFE7002E12
:1031600004D0320001212000FFF792FB002D04D093
:103170002A0002212000FFF78BFB002F04D03A0029
:1031800000212000FFF784FB0134FF2CB0D11EE0AA
:10319000FFF78CFC00250024290000942300220066
:1031A00013200135FFF714FAFF2DF4D1FF2221007F
:1031B000D2002C4804F089FF09E00120FFF75AFEF5
:1031C00005E0002329001A001A20FFF73BFC03202A
:1031D000B5E0FB2B00D0F7E62A68042A00DCEEE617
:1031E0002679E078244B360206439E4200DDEBE66A
:1031F000331D9A4200DCE2E6E35CFE2B00D0E3E6FE
:103200006078A578731E1C2868D007D8082835D0A8
:103210001B285ED0012800D090E007E01E2800D1D6
:103220007EE066D31F2800D180E087E0FF2D00D12B
:1032300084E02800FFF7EAFC67790634B31E290012
:1032400000943A000A20FFF7C3F9064BED00E8505E
:103250005D192F7172E0C046BC0B0020C40B00202A
:10326000C00B0020C41A00203E9B0000BC2200209E
:10327000559B0000509B0000F6030000182D5DD800
:103280006079022813D003281BD0012856D1A71D2E
:103290007A78A479BB78120222431B0413431A00E4
:1032A000FB78AD001B0613435B0003430EE0002BCD
:1032B00044DDB11EA01DFEF7D1FE244BAD00E85049
:1032C0003CE0A379AD005A1E93419B001F4AAB50CE
:1032D00034E0601D1900FFF759FD2FE0FF2D2DD0C0
:1032E0006279022A2AD80634B31E009429000B20E2
:1032F00022E0632B00DD6323002203A8934204DD58
:10330000A118497981540132F7E7D9430022C9173E
:10331000194041180A7001330090290015200BE074
:1033200005340094002229001E2005E0042B05D15D
:103330000022290005340094FFF74AF9701DFFF7B9
:103340003DFA01E0050007E71DB0F0BDBC220020FA
:103350000020704700207047002070470020704711
:1033600001220020054B06491A61585003300431F0
:1033700058508018083158501A607047008000403B
:10338000040500000122034B1A64A822D2009858B9
:103390007047C0460080004010B5FFF7F3FFFA21E8
:1033A000890002F0CDFF10BD10B50100014802F008
:1033B00071FD10BDF010002000487047649B0000B4
:1033C00070B5054E0400335C0D008B4202D002F054
:1033D00089FC355570BDC046CC0F002070B5002467
:1033E000064D635D012B05D10021200002F07AFC1F
:1033F0000023635501341A2CF2D170BDCC0F00208C
:103400000D20704735207047036870B55B100120B0
:10341000052B12D8094A9B009C58094D2B5D002BA7
:1034200005D00021200002F05DFC00232B55200078
:1034300002F002FB01234000184370BD909B000086
:10344000CC0F002070B5036845685C106D1004D483
:103450000B4B9D4202DD1D0000E00025192C0DD80C
:10346000084E335D012B05D00121200002F03AFC0B
:10347000012333552900200002F06CFB70BDC046CB
:10348000FF030000CC0F00200B6870B55D10192DF4
:1034900016D80024012804DD4C68043C62426241D5
:1034A0005400094E735D9C4204D02100280002F0B4
:1034B00019FC7455280002F049FC0423012800D0AF
:1034C0000023180070BDC046CC0F002070B504006A
:1034D0000D0019280ED8084E335C012B04D00121B1
:1034E00002F000FC01233355290020004D1EA941A4
:1034F00002F016FC70BDC046CC0F0020436810B52A
:10350000191F4A424A41006811004010FFF7DEFFD0
:1035100010BD000037B569460200064B684630CB47
:1035200030C11368042B02D100F036FB01E000F03B
:103530005BFB37BD5C9B000010B5084C237D002B66
:1035400005D00021142002F0CDFB002323751420A8
:1035500002F0FCFB43425841800010BDCC0F00201C
:1035600010B5084CA37D002B05D00021162002F0D9
:10357000B9FB0023A375162002F0E8FB4342584133
:10358000800010BDCC0F00207047704710B5034A73
:1035900004210348FFF7B2F910BDC0467C000020AB
:1035A000569A0000E12110B54902094802F0B9FC21
:1035B000FFF7D6FE0A2002F039FA0023FF21054A60
:1035C000995401331A2BFBD100F0AEFB10BDC0465D
:1035D000F0100020CC0F0020F8B50B4E0700300093
:1035E0000D0002F0DDFC041EAC4200DD2C003D00AD
:1035F000EB1B9C4205DD300002F0DCFC287001353D
:10360000F6E72000F8BDC046F010002010B501001C
:10361000014802F08DFC10BDF01000200020704722
:1036200010B51E20FCF7BCFF10BD10B51E20FCF726
:10363000B7FF10BD10B51E20FCF7B2FF002010BD73
:1036400010B51E20FCF7ACFF002010BD10B51E20E9
:10365000FCF7A6FF10BD10B51E20FCF7A1FF10BDA2
:1036600010B51E20FCF79CFF10BD10B51E20FCF706
:1036700097FF10BD10B5034A09210348FFF73EF933
:1036800010BDC0469C000020A89B00000123034AF7
:103690001360034A1068984018437047F00F0020E9
:1036A000F80F00201E2800D91A20084B8000C258AD
:1036B00001239340064A07491360074A1160074AED
:1036C00007491160074A13607047C04694A0000084
:1036D000EC0F00200805005008100020001000200A
:1036E0000C05005018050050F0B5EFF310810123D0
:1036F000194083F31088134E134AB4461268013AF6
:103700009340124A1468124A1568124A002B15D0C9
:10371000166803420BD02660C046C046C046C0466D
:10372000C046C046C046C04616682E6004E06746E4
:103730003E601668084F3E605B08E7E781F310883B
:10374000F0BDC04608050050EC0000200810002025
:1037500000100020EC0F00200C05005030B585B0A3
:1037600001AD0C220649280004F0A6FC0024285DC7
:1037700001210134FFF724FE0C2CF8D105B030BD37
:10378000349C0000F0B53B4C85B0210003220C3185
:10379000684604F091FC210009220F3101A804F0D1
:1037A0008BFCFFF7F9FD344B344CC018236898426A
:1037B00001D2002323602568002D3ED12E006B46E8
:1037C00004339F5D01213800FFF7FAFD0136012126
:1037D000380002F0A5FA092EF1D100266B469F5D54
:1037E00001213800FFF7ECFD01360021380002F01E
:1037F00097FA032EF2D1C82080000138C046C04697
:10380000C046C046C046C046C046C046C046C04688
:10381000C046C046F1D100210520FFF7D1FD0026AA
:103820006B460021985D0136FFF7CAFD032EF7D1E4
:10383000FFF7B2FD1330206019E0FFF7ADFD2368FC
:103840000025984213D3052002F0F6F80C4B0D4EDC
:10385000C01801D4306000E035603068032102F008
:10386000F9FD00230125084A306023601360280019
:1038700005B0F0BD349C000010270000E80F0020C8
:10388000C8FEFFFFF80F0020F00F002010B5012444
:10389000044001D0441002E00D20FCF781FE20001E
:1038A00010BD00007FB5A44E3368002B0BD1A34A96
:1038B0001268002A07D1A24B1B68002B00D139E106
:1038C000FFF760FF36E19F4D2A68002A2AD19C4A03
:1038D0001268002A07D0FFF755FF002800D129E120
:1038E000FFF73CFF05E0954A1268002A01D1002B42
:1038F000F6D1924B19681A00002911D03468002CB7
:103900000ED101AD0C22904928001C6004F0D4FBBC
:10391000285D00210134FFF753FD0C2CF8D109E19B
:103920003368136000210D2002F0FAF900210E2007
:1039300002F0F6F900210F2002F0F2F92E68012EB4
:1039400056D0022E00D19CE0002E00D0ECE00136D3
:1039500031007A4C04202368994302F0E1F90421F4
:10396000236805200B405942594102F0D9F9102132
:10397000236806200B405942594102F0D1F98021B9
:10398000236809010B40594259410C2002F0C8F943
:103990008021236809020B40594259410B2002F053
:1039A000BFF98021236849020B40594259410A203E
:1039B00002F0B6F98021236889020B40594259412F
:1039C000092002F0ADF980212368C9020B40594259
:1039D0005941082002F0A4F9802321681B030B4001
:1039E00059425941072002F09BF931000D2099E01E
:1039F0000221524C072023680B405942594102F0E2
:103A00008FF90820216801400B005942594102F00A
:103A100087F980212368C9000B405942594105208C
:103A200002F07EF98021236849010B405942594137
:103A3000062002F075F980212368C9010B40594224
:103A40005941042002F06CF98021236889030B405E
:103A5000594259410A2002F063F9802321681B046E
:103A60000B4059425941092002F05AF931000C200B
:103A700002F056F931000B2002F052F931000E200D
:103A800050E020212D4C072023680B40594259411A
:103A900002F046F94021236808200B405942594161
:103AA00002F03EF98021236809200B405942594118
:103AB00002F036F98021236849000B4059425941F0
:103AC0000A2002F02DF98021236889000B40594219
:103AD00059410B2002F024F98021236889010B4011
:103AE000594259410C2002F01BF9802123684903F7
:103AF0000B4059425941062002F012F980212368F7
:103B0000C9030B4059425941042002F009F98023AE
:103B100021685B040B4059425941052002F000F92D
:103B200001210F2002F0FCF82B680321581C02F041
:103B300077FD29607FBDC046FC0F0020F40F0020F8
:103B4000F00F002004100020349C0000006810B525
:103B5000C30703D5FFF79AFE054B1860054B1B689A
:103B6000002B03D0024B186800F06AFB10BDC04662
:103B7000FC0F0020101000200022054B10B51A6029
:103B8000044B1B68934201D000F058FB10BDC046A7
:103B9000FC0F00201010002070B505000068FFF732
:103BA00075FE04006868FFF771FE631E0100042BB8
:103BB00014D8451E042D11D805226A43D3180122BA
:103BC00015009D402B00064805682B430360054BFC
:103BD0001B68002B02D0200000F031FB70BDC046F6
:103BE000FC0F00201010002070B505000068FFF7E2
:103BF0004DFE04006868FFF749FE631E0100042BB8
:103C000014D8451E042D11D805226A43D318012269
:103C10009A401300064802689A43064B02601B68EC
:103C2000002B03D00022200000F009FB70BDC0462D
:103C3000FC0F0020101000202C4BF7B51B6804006F
:103C4000002B03D101204042FFF72CFD0126246800
:103C5000344219D0FF226310180212041040FF22D0
:103C6000611212020A40DBB210431843204B1B685A
:103C7000202B06D1B4401F4BA40EA400E358000231
:103C80001843FFF731FD30E0032525402DD1042CEA
:103C90002BD90F2322681340062B26D1FF271309A7
:103CA00001933F04019B9D421FDAAB00E3185A6861
:103CB000324218D0531018023840FF2184460902BE
:103CC000501208406146DBB208431843084B1B689A
:103CD000202B06D15200920E064B9200D3580002C0
:103CE0001843FFF701FD0135DCE7F7BDEC0F0020BD
:103CF000EC000020609C00000B6810B50200D807A3
:103D000001D5581001E0012040421823012A03DDAB
:103D10004A68042A00D10833024A1360FFF7C2FC44
:103D200010BDC046EC000020012010B54042FFF756
:103D3000B9FC0020FFF7D8FC10BD00000068F8B502
:103D4000C30702D5FFF7A2FD0BE0830726D10428A5
:103D500024D90F2203681A40042A1FD11B091DD041
:103D600000790300203B5E2B18D805220020534326
:103D70000B4E9D18043AAB420CD0052110249F5DD8
:103D80003C4200D080180139520064100029F7D15C
:103D90000133F0E701234000184300E00120F8BDA3
:103DA000609D0000F0B5050085B008680C00FFF7C5
:103DB0006DFD0390022D08DD6068FFF767FD0700C9
:103DC000A068FFF763FD040001E00124270005233C
:103DD0006343053B0293012326000193231D9E426A
:103DE00034DC3D003B1D9D422BDC731E042B23D88D
:103DF0006B1E042B20D8029B039A591E019B491964
:103E00001A40204B0AD001228A4019680A431A60DE
:103E10001D4B01221B68002B0ED009E001208840B9
:103E20000100186888431860174B1B68002B03D0EB
:103E30003100280000F003FA019B01355B0001937B
:103E4000D0E7029B013605330293C7E73D1D042DE1
:103E500015D8012C13D126003300AB40094A116854
:103E60009943094B11601B68002B04D0781D002278
:103E7000210000F0E4F901340535062CECD105B041
:103E8000F0BDC046FC0F00201010002010B5034A02
:103E900001210348FEF732FD10BDC046E4000020BA
:103EA0004C9C00000120704710B5064C200000F02B
:103EB000FFFA0549200000F01FFB0122034B1A60A6
:103EC00010BDC04634100020801A06000C100020DF
:103ED00010B501210D20FFF773FA01210E20FFF725
:103EE0006FFA00210F20FFF76BFA044C200000F05E
:103EF0001BFA1021200000F033FA10BD2010002022
:103F000010B504680D20E30703D56410FF2C03D916
:103F10001720FCF745FB06E0FFF7DAFFE1B20248A5
:103F200000F040FA002010BD2010002010B5FFF76F
:103F3000CFFF0021034800F035FA01234000184369
:103F400010BDC0462010002010B5034A07210348C9
:103F5000FEF7D4FC10BDC046F00000203B9F0000DF
:103F6000F8B5012306681E4205D045681D4202D0FF
:103F700084681C4201D10D2004E076106D10802E63
:103F800003D91520FCF70CFB1DE01620FF2DF9D8F6
:103F900064101720FF2CF5D80B4B1B68002B01D1A8
:103FA000FFF782FF094FF1B2380000F02DFBE9B2B4
:103FB000380000F03EFAE1B2380000F03AFA38007A
:103FC00000F08CFB0020F8BD0C1000203410002005
:103FD000F7B501242300A04237DD0A68144234D02B
:103FE0001B4B55101B684C68002B01D1FFF75CFF81
:103FF0000127184EE9B2300000F006FB3C4205D024
:104000003C413000E1B200F014FA1AE003252540EB
:1040100017D1042C15D90F2322681340062B10D179
:1040200013090193019B9D420BDAAB00E318596819
:10403000394204D04910C9B2300000F0FAF9013514
:10404000F0E7300000F04AFB00231800FEBDC04638
:104050000C10002034100020144B70B51B680500B4
:104060000E00002B01D1FFF71FFF114CEDB229000C
:10407000200000F0C9FAF1B2200000F0DAF90021C6
:10408000200000F0CDFA002801D040420CE00122CF
:104090002900200000F0B3FA200000F0C0F9002849
:1040A000FAD0200000F0C0F970BDC0460C1000200E
:1040B0003410002010B501240368234202D0416867
:1040C000214201D10D2004E058104910802803D965
:1040D0001520FCF765FA07E0FF2901D91620F8E75B
:1040E000FFF7BAFF4000204310BD10B5072118208C
:1040F000FFF7B2FF7F2801DD0138FF3803007F336F
:1041000001DA7F20404264237F215843494202F074
:10411000A1F9012340424000184310BD10B5082109
:104120001820FFF799FFC30F18180123401015300E
:104130004000184310BD10B505211820FFF78CFF73
:104140007F2801DD0138FF3803007F3301DA7F204B
:10415000404264237F215843494202F07BF9012306
:104160004000184310BD10B503211820FFF774FF5D
:104170007F2801DD0138FF3803007F3301DA7F201B
:10418000404264237F215843494202F063F90123EE
:104190004000184310BD0000F8B501263400B042BD
:1041A00036DD0F683E4233D04D68AB0730D1042D69
:1041B0002ED90F232A681340062B29D1154B1B68D3
:1041C000002B01D1FFF770FE0024354204D12B688B
:1041D0001C09202C00D920240F4E7F10F9B2220098
:1041E000300000F00CFAA700EF19AF420DD03000FC
:1041F00000F015F90028FAD0300000F015F901237D
:104200004000184368600435EFE701206400044370
:104210002000F8BD0C100020341000200020704752
:104220000020704700207047002070470020704732
:10423000002070470020704700207047704770478B
:104240007047000010B5034A08210348FEF756FBEB
:1042500010BDC046280100207C9F000010B5FFF76C
:10426000A1F9AF20C000FDF79BFEFEF7B9FB0448A3
:10427000FEF70CFDFEF710FAFEF774FD10BDC04608
:10428000169B000010B5FDF71DFE10BD70B5002592
:1042900004AC24780573A94205D10A4B0A4A2321AC
:1042A0000A4803F089FE01600949920052589B00B8
:1042B00002715B588371A3005B58856043710223D0
:1042C000C37170BDFF9F0000C29F00000DA00000E1
:1042D00094A00000037B002B04D14373837303611C
:1042E00001330373704700001FB50191A021002422
:1042F0000068C900D2B24450012A07D0A24203D0BC
:10430000032A05D1042202E0022200E00622134320
:10431000034A8350034B019AC250012343501FBDEF
:10432000540500002405000010B50400FFF7D2FF7B
:10433000A1222368A179D20099506179064A200010
:104340009950217904329950044B19685A689B6836
:10435000FFF7CAFF10BDC0460C0500001410002076
:104360004BB2002B0CDB80233F290CD81F290CD823
:104370000F290CD807290CD803290CD81B060BE0F1
:1043800080239B0408E0DB0406E01B0504E05B05DA
:1043900002E09B0500E0DB050168014A8B50704795
:1043A000240500000368074A99501A00FC32D168BE
:1043B0000029FCD0A321C90058580023C0B2D36003
:1043C0007047C0461C05000007B58022074BD20588
:1043D0001A6000229A6002321A7111230E32009381
:1043E000034905330348FFF751FF07BD14100020B0
:1043F0000030004020100020F8B505000E00170026
:104400000024BC4208D02B68315D1B682800984707
:10441000002801D00134F4E72000F8BD704710B542
:104420001C3001F063FD10BD10B51C3001F050FDD3
:1044300010BD70B5437E0D00002B05D06430040024
:1044400001F063FD002801D0002004E020002900D5
:1044500001F02FFD012070BD10B51C3001F04CFDA6
:1044600010BD0000F7B50193FA23002504009B005E
:1044700083600D4B4560083303601C300F0016004D
:1044800001F00CFD2000643001F008FD074AB60081
:10449000B35827616375019B20009B009B5865768C
:1044A000A576A375FEBDC04674A0000094A00000D0
:1044B0000123A022C375837D0C49C133FF33D2058C
:1044C0009B009950437DC133FF339B009950CC2111
:1044D0000369074A490499500521243A9950817D7E
:1044E00008329950417D034A995070470C060000EC
:1044F000240500000C050000A02302690020DB0059
:10450000D0500948814204D90848814204D9CD21BC
:1045100003E0CC21490401E08021C9040448115082
:104520000521D1507047C046A086010090D00300FD
:1045300024050000F7B5050000200C00019382421D
:104540005CD0161E402E00D940262F001C373800A4
:1045500001F0BAFCB1222B69D20080219C500122CB
:1045600089005A50A97E002901D11A621A600024DC
:10457000731E2A69A34206D1019B002B03D080231E
:1045800002219B00D150012313621300FC33D96830
:10459000002902D1996A0029F9D0996A00290AD123
:1045A000D960A323DB00D1583800C9B2013401F02F
:1045B00080FCA642DCD8019A2B69002A04D11A009B
:1045C000FC32916A00290AD001210022AA765961A1
:1045D0001900FC3188680028FCD08A6007E00121BE
:1045E000A976D961D16C0029FCD00021D164FC33BB
:1045F0009A6A002A01D000229A62E0B2FEBD10B58C
:104600000123FFF797FF10BD0300AC3310B5040082
:104610001970643001F058FC0123637610BD00006E
:10462000F8B500220D0001004276AC3103690400A8
:104630000878B121C9005850802189005A500132B0
:104640001A629A6026006436300001F04FFC0028A0
:104650000ED03000276901F03BFC1E4BF850236957
:10466000FC331A6A002A0CD19A6A002AF9D008E0B1
:104670002369002D0AD11A00FC32916A002905D164
:104680000EE09A6A002AF3D11A62DBE701225A612E
:104690001A00FC3291680029FCD00021916006E0EC
:1046A0000121D961D16C0029FCD00021D1641A000C
:1046B0000020FC32916A81420BD0074990625A581F
:1046C00002305A50824204D0043A534253410230DD
:1046D000C01AF8BD1C050000C404000010B501217B
:1046E000FFF79EFF10BD000010B5132312220249F0
:1046F0000248FFF7B7FE10BD004000403410002014
:1047000030B5214A4B0087B05B0893421EDD1F4A3B
:10471000934205DD02000B0003F010F807B030BD36
:1047200002AA00F035F803231840049A059B0128DB
:104730001ED0022811D000281FD00298039900F043
:104740002DFA80231B069C466144E7E700230022E4
:104750000093002300F088FFE0E70124029803990A
:10476000009400F081FF80231B069C466144D5E73E
:104770000298039900F012FAD0E7012402980399F5
:10478000009400F071FFC9E7FB21E93FFFFFEF7FD5
:10479000F0B54E4657464546E0B4DC4B4E0090B06F
:1047A0001700894676089E4200DC81E0D84B9E4285
:1047B00020DCD84A002900DC89E1D74B02F0BEFF9B
:1047C000D54B04000D009E4200D18AE0D34AD44B61
:1047D00002F0B4FF02000B0020003A607B60290069
:1047E00002F0ACFFCD4ACE4B02F0A8FFB860F960F2
:1047F000012066E0CB4B9E4200DC8DE0CA4B9E421E
:1048000065DCCA4932158A46924453461B05F51A9F
:104810002900040003F0E6FA03F01AFB02000B0083
:10482000200029000A920B9302F088FF0022C04B5F
:1048300002F00AFD0290039103F0D4FA03F008FBA2
:1048400004000D0002000B00029803990C940D95D2
:1048500002F074FF0022B64B02F0F6FC00220023A7
:104860000E900F9101F000FF002800D14CE10023D1
:1048700000222000290001F0F7FE0222431E984189
:10488000131AAC4A3900019202220AA80092524639
:1048900000F09EFA4B46002B13DA80221206944653
:1048A0007B68404263447B60FB686344FB6008E0D4
:1048B00002000B003A607B60002200230020BA60F7
:1048C000FB6010B01CBC90469946A246F0BD0200A9
:1048D0000B0002F033FFB860F960386079600020A7
:1048E000EFE7D3228E4B520502F028FF924A934BFA
:1048F00004000D0002F022FF02000B0020003A60CD
:104900007B60290002F01AFF8B4A8C4B02F016FFE5
:10491000B860F9600120D4E700F056FF884A894B5F
:1049200004000D0002F090FC0022874B02F052F8C8
:1049300003F058FA804603F08BFA764A764B0690DD
:10494000079102F081FC02000B002000290002F018
:10495000F5FE734B02900391069807996F4A02F097
:1049600073FC434604000D00049405951F2B30DCB6
:10497000013B764A9B009B589E422AD002000B00C6
:104980000298039902F0DAFE02000B0005000C0009
:104990003A607B60029803992A00230002F0CEFE61
:1049A000049A059B02F0CAFE06000B003200BA60B2
:1049B000FB604B464046002B00DB82E780231B0652
:1049C0009C46644461443D607C60BE60F960404246
:1049D00077E7049A059B0298039902F0AFFE0B005B
:1049E00002003A607B604B0036155B0D05000C0041
:1049F000F31A102BCEDD06980799D322484B5205A7
:104A000002F022FC04000D0002000B000298039942
:104A100002F094FE02000B00029803990892099399
:104A200002F08CFE22002B0002F088FE04000D0034
:104A300006980799404A414B02F006FC22002B00E1
:104A400002F07CFE02000B00049005910898099981
:104A500002F074FE02000B003A607B604B005B0DBD
:104A6000F61A0500089A099B0C0002920393312E56
:104A700090DD06980799B822304B920502F0E4FBCE
:104A800004000D0002000B000298039902F056FE8C
:104A90000A0001001300029103920200089809998C
:104AA00002F04CFE22002B0002F048FE04000D0034
:104AB00006980799264A274B02F0C6FB22002B00D6
:104AC00002F03CFE02000B000492059358E7124BE3
:104AD00001F080FF104B04000D009E423CD00F4AB5
:104AE0000F4B01F077FF02000B0020003A607B6063
:104AF000290002F023FE094A094B01F06BFFB86060
:104B0000F96001204042DCE60323BAE6FB21E93FDD
:104B10007BD9024000004054FB21F93F3163621A07
:104B200061B4D03DFB213941FFFFEF7FEAFBFFFF7E
:104B30000000704190A100007370032E8A19A33BFE
:104B400083C8C96D305FE43F0000E03F10A1000062
:104B5000C14920259A837B39D3220D4B520501F0A0
:104B600039FF0C4A0C4B04000D0001F033FF02002A
:104B70000B0020003A607B60290002F0DFFD054A4F
:104B8000054B01F027FFB860F9600120404298E62C
:104B900061B4D03D7370032E8A19A33BF0B54F4624
:104BA0004646C0B487B000920193754B4F008146D2
:104BB00088467F089F4263DC03F014F9002800D187
:104BC000DAE04A4643464846414602F03DFB0400CF
:104BD0000D006C4A6C4B02F037FB6C4A6C4B01F0D9
:104BE000F9FE22002B0002F02FFB6A4A6A4B02F00A
:104BF000A5FD22002B0002F027FB684A684B01F05C
:104C0000E9FE22002B0002F01FFB664A664B02F011
:104C100095FD22002B0002F017FB644A644B01F063
:104C2000D9FE22002B0002F00FFB0290039100221C
:104C3000604B2000290002F007FB029A039B06004C
:104C40000F002000290002F0FFFA009A019B0400E7
:104C50000D004846414602F0F7FA02000B00200022
:104C6000290002F06BFD02000B003000390002F059
:104C700065FD02000B0000204F4902F05FFD70E06F
:104C800002000B0002F0E0FA04000D003D4A3E4B2A
:104C900002F0DAFA3D4A3E4B01F09CFE22002B0066
:104CA00002F0D2FA3B4A3C4B02F048FD22002B00B6
:104CB00002F0CAFA394A3A4B01F08CFE22002B006E
:104CC00002F0C2FA374A384B02F038FD22002B00BE
:104CD00002F0BAFA354A364B01F07CFE2B00220076
:104CE00002F0B2FA354B029003919F429FDD344BA4
:104CF00000229F423ADC334900207B182E491600DF
:104D00001F0002F01BFD049005910022294B20009A
:104D1000290002F099FA32003B0002F00FFD029ADE
:104D2000039B06000F002000290002F08DFA009A74
:104D3000019B04000D004846414602F085FA02003E
:104D40000B002000290002F0F9FC02000B003000EB
:104D5000390002F0F3FC02000B000498059902F000
:104D6000EDFC07B00CBC90469946F0BD164B0026F2
:104D700004920593154FC8E700200F49F1E7C0469C
:104D8000FFFF3F3ED43888BEE9FAA8BDC4B1B4BD28
:104D90009EEE213EAD529C804F7E923E9015CB19E7
:104DA000A001FA3E7751C1166CC1563F4C5555557E
:104DB0005555A53F0000E03F0000F03F3233D33FA0
:104DC0000000E93F0000E0FF0000E73F0000D23FA5
:104DD000F0B556464D4644465F46F0B48E4CA54469
:104DE000099119001400A89A0B938C4B9200D25889
:104DF0000B000290013BE01E18211D0016000892D6
:104E0000009301F027FBC3430200DB171A40130095
:104E1000110001330E929A009B1ADB001B190693B6
:104E20004C1B761918D4A99BA5009C46361926AFB1
:104E30006544013607E0286803F00AF8013403C727
:104E40000435B44208D0002CF5DA002000210134EA
:104E500003C70435B442F6D1089B002B01DA00F0F9
:104E6000F9FB76AB19008B4626AA9146089A0A935D
:104E70000132D2009344029A9A469046009BDB008E
:104E8000994408339844009B002B00DAB5E14C4666
:104E900000260027029D2268636803CD02F0D4F942
:104EA00002000B003000390001F094FD083C0600C0
:104EB0000F004545EFD15346C0C39A4608239C4690
:104EC000E144DA45DFD10899554A0B009446634422
:104ED0009B0012A884461A000298624483460D92F1
:104EE0000B9A0433D200634493440F930591059ABF
:104EF0000A98D30019000C938C46030063441E6883
:104F00005F68002A34DD12AB99461300454A80469B
:104F100094466344DB00984474AB9A460022424BAB
:104F20003000390002F090F902F05CFF02F090FFCF
:104F300000223E4B04000D0002F086F902000B0037
:104F40003000390002F0FAFB02F04CFF4B4601C37F
:104F50009946434620001A685B68290001F03AFD33
:104F600008235B429C46E04406000F00D045D5D1A3
:104F7000069B30001A003900994600F0C1FCFF235F
:104F800000229B0504000D0002F05EF900F020FCF9
:104F90000022274B02F058F902000B0020002900E4
:104FA00002F0CCFB04000D0002F01CFF804602F072
:104FB0004FFF02000B002000290002F0BFFB4C460F
:104FC00006000F00002C00DCF8E0059B18205A1E9C
:104FD000920012AB9B58001B19000141884481408C
:104FE0005B1A12A98B501722121B13410793079BC0
:104FF000002B4BDD01239C46059BE044002B00DC8D
:10500000F2E280251096119712AB00210024094886
:105010006D04059F19E0C04684FDFFFF98A20000C3
:10502000FEFFFF3FFFFFFF1F0000703E00007041CA
:1050300000002040FFFFFF00002A02D0AA1A1A60D9
:105040000134013104338F4209DD1A68002CF3D09A
:10505000821A01311A60012404338F42F5DC109E5C
:10506000119F069B002B0EDD012B00D1B1E0022B1E
:1050700009D1059B12A95A1E920012AB9B5810939E
:105080009B029B0A8B50079B022B7ED000230022A1
:105090003000390001F0E8FA059B002800D16BE2EE
:1050A00008995A1E914210DCBF490F988C4612A9EC
:1050B00063448C4600219B0063441C68043B2143ED
:1050C0008342FAD1002900D0B5E0089B12AA013B27
:1050D0009B00D358002B00D084E201220D9B043B9F
:1050E000596801320029FAD005990B008C4601332A
:1050F00062440792934242DC0E9A9446A99A634412
:1051000092460B9A9B00944626AA90469A44059B89
:105110000A9A6344DB0098440C9B94469946079B8B
:10512000E144DB00634405935346186802F090FEA7
:10513000434618605960009B002B23DB4446002641
:105140000027029D2268636803CD02F07DF802000B
:105150000B003000390001F03DFC083C06000F0058
:105160005D45EFD14B469E60DF6004239C460433CF
:10517000E2449C46059BE144E0449945D4D1079B19
:105180000593B4E600260027ECE732003B00002040
:10519000864902F0D3FA06000F00002C00D175E713
:1051A000069A0020814900F0ABFB02000B003000A2
:1051B000390002F0C3FA06000F0067E7069B002BD8
:1051C00012D1059B12AA013B9B00D558EB15079302
:1051D0000DE7059B12A95A1E920012AB9B58109323
:1051E0005B025B0A8B504EE70022714B01F060FAC4
:1051F00000280ED10023079348E7534600260027D6
:10520000C0C39A4608239C46E144DA4500D03AE6FA
:1052100059E601239C4601330793059BE044002B8C
:1052200000DDEEE632003B000020604902F086FA25
:1052300006000F002AE743460B93069B12A8183B73
:10524000190006939300C3580092002B0FD15648C3
:105250001300844612A8634484469B006344043BC5
:105260005868013A18390028F9D000920691069A38
:1052700000204E4900F044FB009B04000D00002B71
:1052800000DAB3E112AA94469F00DB0067449C4613
:105290000A9A0593624493461600386802F0D8FDD6
:1052A00022002B0001F0D0FF424B306071600022E1
:1052B0002000290001F0C8FF083E74AB04000D0077
:1052C000043FB342E9D100239A464EAB0293089BB8
:1052D00099464B4600260027002B21DB8020364BC9
:1052E0005D469846C005354900260027002408E0A1
:1052F00008239C460835E044A24511DB4346186864
:1053000059682A686B6801F09FFF02000B003000AB
:10531000390001F05FFB013406000F00A145E7DA18
:10532000029A53469446DB0063441E605F6001238B
:105330009C46093BE2449C4674ABE3449B45C8D180
:10534000029B9946A89B022B00DD82E0002B37DCF4
:105350001DD1059B00254B441E0000243268736854
:105360002800210001F036FB009B05000C00083EE0
:105370005A1E0092F2D2079B002B03D080231B06FB
:105380009C4664442A00230009990A604B60072068
:105390000B9B18409F239B009D443CBC9046994624
:1053A000A246AB46F0BDC046FFFFFF3F0000F03F06
:1053B0000000E03F0000703EA8A20000FB21F93F82
:1053C000059B00204B441E0000214CAF32687368DF
:1053D000083E01F0FFFABE42F8D1079B002B24D013
:1053E0008023099A1B06CB18106053600B00020043
:1053F0004E984F9902F0A2F9009B002B0BDD01247F
:1054000050AD0CCD01F0E6FA009B0134A342F8DA6E
:10541000079B002B03D080231B069C4661440B0096
:10542000020009998A60CB60B1E702000B00099C79
:10543000226063600B0002004E984F9902F07EF9E3
:10544000009B002BDBDC0B00020009998A60CB601B
:105450009DE7A89B032B9AD1009B002B00DCE3E087
:105460007E4A059B94464B441E685F68009B6344DC
:105470009A46DB004B4498464CAB9B4643465C68DF
:105480001B681800210032003B000290039101F0DC
:10549000A1FA04000D0002000B000298039902F02B
:1054A0004DF93B00320001F095FA43469860D9600F
:1054B0001C605D6008235B429C46E04426002F0090
:1054C000C345DBD1009B012B00DCADE0059BC8464A
:1054D0004B441E685F685346DB009B46D8444346F6
:1054E00030005C681B683900009301941A002300A7
:1054F00001F070FA04000D0002000B000098019901
:1055000002F01CF93B00320001F064FA4346986057
:10551000D9601C605D6008235B429C46E044260025
:105520002F00C145DBD15D460027002408354D44DE
:1055300050AE2A686B683800210001F04BFA083D34
:1055400007000C00AE42F4D1079B002B71D0099AE2
:105550004E994B461160802109068C465B6849468E
:10556000634453604B46DB688968634464449160DC
:10557000D360176154610AE7994643460B93069B33
:1055800030005A42390000F0BBF90022344B0400CD
:105590000D0001F08DF8002832D0324B002220009F
:1055A000290001F051FE02F01DFC4A46060097005A
:1055B00002F04EFC00222A4B01F046FE02000B00D6
:1055C0002000290002F0BAF802F00CFC12AAD05117
:1055D0004A46069B0132183300920693930012AAA2
:1055E000D65044E601227FE500243AE5A89B022B31
:1055F00014DC002B0FDC00D0C9E600250024BAE63D
:105600004B46200029009E0002F0ECFB12AB9851A3
:105610004B4600932BE600200021DEE64EAB994678
:10562000A89B032B00D0B2E6079B00270024002B89
:105630008DD14E9A4F9B09990A604B604B469A68F0
:10564000DB68009201938A60CB603A0023000A6114
:105650004B619CE676AB0A9335E4C046FFFFFF1F23
:10566000000070410000703EF0B54F464646C0B4A1
:1056700087B000920193464A4B00814688465B08FA
:10568000934205DC02F0AEFB4146031E484666D05D
:105690004A4643464846414601F0D6FD04000D0007
:1056A00002000B004846414601F0CEFD394A3A4B14
:1056B00006000F002000290001F0C6FD374A384BD4
:1056C00002F03CF822002B0001F0BEFD354A364BBB
:1056D00001F080F922002B0001F0B6FD334A344B73
:1056E00002F02CF822002B0001F0AEFD314B324AC3
:1056F00001F070F90E9B02900391002B34D00098BA
:10570000019900222D4B01F09FFD029A039B04900A
:1057100005913000390001F097FD02000B0004985C
:10572000059902F00BF822002B0001F08DFD009A84
:10573000019B02F003F8224A04000D00214B3000C7
:10574000390001F081FD02000B002000290001F06A
:1057500041F902000B004846414601F0EFFF07B057
:105760000CBC90469946F0BD02000B0020002900B9
:1057700001F06AFD124A134B01F0E0FF32003B00DA
:1057800001F062FD4A46434601F024F9E7E7C046CE
:10579000FFFF3F3E7CD5CF5A3AD9E53DEB9C2B8AA3
:1057A000E6E55A3E7DFEB157E31DC73ED561C119FE
:1057B000A0012A3F1111813FA6F810110000E03F1F
:1057C000495555555555C53F49004B081900704777
:1057D000454AF8B5564692464B005B0D9A444D46F5
:1057E0005F4644465246F0B4894605000C000E0060
:1057F0000700132A22DC002A47DB52463B4B1341A9
:1058000098460B0042461340034311D0384A394BA7
:1058100001F0E0F80022002300F040FF002805D04E
:10582000002C41DB4E46434600279E4338003100A2
:105830003CBC90469946A246AB46F8BD5246332A38
:1058400008DD8023DB009A45F2D102000B0001F055
:10585000C1F8EDE7284A9446012263445242DA40F7
:1058600093460242E4D0224A224B01F0B3F80022D0
:10587000002300F013FF0028D8D0002C1ADB5B4671
:105880004E469F4338003100D2E7194A194B01F0C8
:10589000A1F80022002300F001FF0028C6D0002C50
:1058A00016DB00270026C1E7802352465B03134125
:1058B0009944B7E75346142B12D03423524601279C
:1058C0009B1A9F407F19AF429B415B429944D6E7A8
:1058D0006400640825430027002DA7D0074EA5E7E4
:1058E000133B9C46E144CAE701FCFFFFFFFF0F00AA
:1058F0009C7500883CE4377EEDFBFFFF0000F0BFA5
:105900004B0070B55B0D14000A00002B1AD14B0040
:105910005B08034315D00022224B01F095FC224B7B
:105920000A009C4222DB4B005B0D363B1F4DE31807
:10593000AB4220DC002B0DDD1D4C1B0522401A4321
:10594000110070BD1B4DAB42F0D102000B0001F005
:1059500041F8F6E71D00353518DA174B02009C4276
:105960000ADC0B001548164900F032F8134A144BB4
:1059700001F06AFCE5E702000B001248124900F052
:1059800027F8104A104B01F05FFCDAE7084C363379
:1059900022401B051343190000220C4B01F054FC5C
:1059A000CFE7C04600005043B03CFFFFFE070000B9
:1059B000FFFF0F80FF07000050C3000059F3F8C23B
:1059C0001F6EA5019C7500883CE4377E0000903C6A
:1059D00030B54A00DB0FDB0752081A43110030BD17
:1059E00003210A4802680A430260094802680A4320
:1059F00002600849084A094B9B1A03DD043BC8585A
:105A0000D050FBDC00F0B4F9FAF7B4FB24050040F9
:105A1000540500407CA50000000000203402002056
:105A2000FEE7FEE7FEE7FEE7FEE7FEE7014B186054
:105A30007047C04670010020F7B500231E2877D8B4
:105A40003C4B8000C258042A14D006D8022A0DD03C
:105A50000ED80423012A14D069E0062A0ED00BD3F5
:105A60001A2A0DD002231B2A0BD060E0082308E07D
:105A7000102306E0202304E0402302E0802300E01E
:105A800001232D4A1268082A04D9092A05D00A21BF
:105A9000022404E00821002401E011000124A025D3
:105AA00001261C272548ED004651254D254E2D6821
:105AB0001B02AD003D400195234D2D680095855991
:105AC000AC466746214D3D401D4385518359C02555
:105AD0009C46009BAD021D40FF2367461B023B40D6
:105AE0002B43019D1D43009B5F0160231F402B0042
:105AF0003B431C4301238451154C036063680F48EA
:105B0000002BFBD00024124B01255C60A123DB009D
:105B1000C3584560A025ED0044511BB2914207D007
:105B200002D98A1AD34003E0521A934000E00023BE
:105B30001800FEBD94A00000740100200070004019
:105B40006C0100200405000068010020FF00FFFF39
:105B5000FC700040F0B51E286CD8374B8000C2584E
:105B6000364B1E68002E2ED1C2243548A40007599A
:105B7000344B03253B40C0273F023B430351802366
:105B8000893C9B00FF3C03512F4F03602F4B803C0F
:105B9000D859FF3CA043D8510437D859A8432043D3
:105BA000D8510837D8590C35A843083D2843D85157
:105BB000A820C0001E508026C120760280001E5002
:105BC0001C601E4B1C6000231426214834005C43DB
:105BD000255804006F1C0FD1142058432250A020D8
:105BE0000325C132FF329200C0051550194A080042
:105BF0001268082A03D10BE0AA4218D1ECE7082A60
:105C000002D9083AD14002E00820821A91400800E7
:105C100014225343E3189A680C495132FF32920020
:105C200058605050DA68C1239B00CA5002E001332B
:105C3000032BCBD1F0BDC04694A00000EC10002097
:105C400000E100E0FF00FFFF0405000000900040BD
:105C500078010020700100201E4BF0B5596C18002F
:105C60001D4A002914D0A025A12600230124ED05FA
:105C7000F600D1584F1C06D0D7187F68002F02D0ED
:105C800027008F40AF5114333C2BF2D100234364E3
:105C9000131DA02540329446002001240F4EED052F
:105CA000DA680F49920057180A495218526C002AB4
:105CB0000CD01A1F1268511C05D01968FF2902D098
:105CC00021009140A9513A00FC32506414339C45A4
:105CD000E6D1F0BDFC900040780100200C050000EA
:105CE0000090004000B51E2816D80C4A83009B582F
:105CF000032911D8A0220800C133FF33D2059B002D
:105D000000F014FB02080406002104E00C2102E06C
:105D1000042100E00321D15000BDC04694A0000042
:105D20001E280DD8074B8000C058A0220123D205A1
:105D30008340002901D1044901E0A121C900535049
:105D40007047C04694A000000C050000030000202E
:105D50001E2B0AD8A222A021D200C9058858034AC6
:105D60009B009B58D84001231840704794A0000026
:105D70002D4B10B51A78012A19D12C4A1268120736
:105D800015D12B4AE0241168F0220800104021426E
:105D90000BD128490968114209D12749274A1160C6
:105DA0008021274A0902116001E03028F1D01A78D9
:105DB000012A0DD11D490968090709D1F0201C49A4
:105DC00009680140402903D11A490968014223D0DA
:105DD0001B68DBB2012B25D1144B1B681B0721D19B
:105DE000134B1A68F0231A40A02A04D1114A1268F2
:105DF0001A4203D016E0D02A14D1F7E7114B1A68E3
:105E0000012A03D1C022104B1A600BE00F4A1A601E
:105E10001A68012AFCD1F5E7C1218020C900C0051C
:105E20004250D5E710BDC046E00F00F0E40F00F08F
:105E3000E80F00F0EC0F00F0DFFF07C004050040A2
:105E4000186C004000EC064014EC0640759300000E
:105E5000F7B506000D000C008B180193019B671B22
:105E60009C4207D0336821781B6830009847013482
:105E70000028F3D13800FEBD70B505000C00081EE7
:105E800007D002F04FFD2B6802005B68210028005C
:105E9000984770BD10B5FFF7EFFF10BD10B5402259
:105EA0000021040002F011F9002320002364636440
:105EB00010BD3F23026C10B5541C2340446C9C421F
:105EC00001D08154036410BD002303644364704710
:105ED000436C026C934206D03F21C25C01330B40FD
:105EE0004364100001E0012040427047036C406CA5
:105EF000181A00D540307047436C026C934201D0B1
:105F0000C05C01E0012040427047036C406C5A1CA9
:105F10003F231340181A42424241D0B27047012039
:105F2000704710B503681322DB69984710BD7047AE
:105F30000369054A9950FC331A6A002AFCD00022F2
:105F400001201A627047C0461C050000030010B50E
:105F50005C331A781F2313400122110099400D4B26
:105F60000424D967C221036989005C505A60DA6051
:105F7000A0220021D20099500122074952425A50D2
:105F8000064914305A500C395A5008315A50FFF70C
:105F90009BFF10BD04E100E00C05000014050000AB
:105FA00010B51430FFF7A2FF10BD10B51430FFF785
:105FB000A3FF10BD10B51430FFF78AFF10BD00001D
:105FC000030070B55E331C780269604BD450030047
:105FD0005D331C785E4BD450030061331C785D4BFD
:105FE000012C0CD105005F352E78A225ED0056510D
:105FF000050060352E78A125ED00565100E0002403
:10600000D4509623DB00994238D996231B0199423C
:1060100037D996235B01994236D996239B01994241
:1060200034D9E1239B01994232D99623DB0199426D
:1060300031D9E123DB0199422FD996231B029942E2
:106040002DD9E1231B0299422BD996235B02994259
:1060500029D9E1235B02994227D9E1239B02994286
:1060600025D93D4B994224D9E123DB02994223D91A
:10607000E1231B03994221D8384B21E09E23DB0208
:106080001EE09D231B031BE0354B19E0354B17E049
:10609000EC239B0314E0344B12E0344B10E0344B00
:1060A0000EE0344B0CE0344B0AE0344B08E0344B48
:1060B00006E08023DB0403E0324B01E080235B0534
:1060C0003149002453500423243953501100FC312A
:1060D000CC600C62C1210134890014605C30946092
:1060E000535003781F202200D9B2084082408034E8
:1060F0002648FF345BB20251002B13DA0F230B400A
:10610000083B234C9B089B001B1903242140A14002
:10611000FC348C40DD69A543C0248C402100294318
:10612000D96111E0194C9B089B001B1903242140E5
:10613000A140C025FC348C40AD005E59A643C0246C
:106140008C40210031435951026070BD0C050000A4
:10615000140500006C05000090D0030000D0BE0EB6
:1061600000B013000050270000A04E0000F07500A2
:1061700000509D0000F0EB0000903A0100E0D701D4
:1061800000B0AF0300705F072405000000E100E0ED
:1061900000ED00E0F7B5009308AB1B7800250193F4
:1061A000FA2304009B0083600E4B456008330360B4
:1061B00014300F001600FFF771FE23005C332761D7
:1061C0001E70009B084A9B00995823005D3319708C
:1061D000019B20009B009A5823005E33DD701A70EB
:1061E000FEBDC046E8A2000094A00000036910B5FF
:1061F0001A00FC32D2680400002A0AD0A322D2007E
:1062000099581430C9B2FFF754FE00222369FC33B9
:10621000DA6010BD10B50248FFF7E8FF10BDC046B8
:10622000F01000201D2307B502220093024901331C
:106230000248FFF7AFFF07BD00200040F01000202C
:106240007047000010B500F047F8FFF7F9FF012094
:1062500000F024F8FEF702F8FEF714F8024B002BCA
:10626000FAD000E000BFF7E700000000084A094943
:10627000094B10B51B688858FA22190A1B061843E7
:106280009200002300F01EFA4904C00B084310BD21
:1062900004050000001001405411002070B5041ED8
:1062A00009D0FFF7E3FF050000F014F8FFF7DEFF69
:1062B000401B8442F8D870BD0022044B9A60044A07
:1062C00013680133DBB213607047C046FC10014015
:1062D0005411002070470000C421114A8900505811
:1062E000104B0340C02000020343535080239139D8
:1062F0009B02FF39535013608023A3220021DB054A
:10630000D20099500122A1209A60074BC000195079
:10631000C120023180001950403019501A60704776
:1063200000E100E0FF00FFFF0010014002B47146F1
:1063300049084900095C49008E4402BC7047C046C8
:10634000002243088B4274D303098B425FD3030AB4
:106350008B4244D3030B8B4228D3030C8B420DD3C7
:10636000FF22090212BA030C8B4202D31212090255
:1063700065D0030B8B4219D300E0090AC30B8B4293
:1063800001D3CB03C01A5241830B8B4201D38B0341
:10639000C01A5241430B8B4201D34B03C01A5241E6
:1063A000030B8B4201D30B03C01A5241C30A8B4229
:1063B00001D3CB02C01A5241830A8B4201D38B0214
:1063C000C01A5241430A8B4201D34B02C01A5241B8
:1063D000030A8B4201D30B02C01A5241CDD2C3092A
:1063E0008B4201D3CB01C01A524183098B4201D3A6
:1063F0008B01C01A524143098B4201D34B01C01A91
:10640000524103098B4201D30B01C01A5241C30808
:106410008B4201D3CB00C01A524183088B4201D377
:106420008B00C01A524143088B4201D34B00C01A63
:106430005241411A00D20146524110467047FFE7CF
:1064400001B5002000F0F0F802BDC0460029F7D0E9
:1064500076E7704703460B437FD4002243088B4204
:1064600074D303098B425FD3030A8B4244D3030BDB
:106470008B4228D3030C8B420DD3FF22090212BAA0
:10648000030C8B4202D31212090265D0030B8B421C
:1064900019D300E0090AC30B8B4201D3CB03C01A06
:1064A0005241830B8B4201D38B03C01A5241430BE1
:1064B0008B4201D34B03C01A5241030B8B4201D3D1
:1064C0000B03C01A5241C30A8B4201D3CB02C01A3C
:1064D0005241830A8B4201D38B02C01A5241430AB4
:1064E0008B4201D34B02C01A5241030A8B4201D3A3
:1064F0000B02C01A5241CDD2C3098B4201D3CB014A
:10650000C01A524183098B4201D38B01C01A5241F8
:1065100043098B4201D34B01C01A524103098B42FC
:1065200001D30B01C01A5241C3088B4201D3CB00E7
:10653000C01A524183088B4201D38B00C01A5241CA
:1065400043088B4201D34B00C01A5241411A00D27A
:1065500001465241104670475DE0CA0F00D04942E3
:10656000031000D34042534000229C4603098B4253
:106570002DD3030A8B4212D3FC22890112BA030ADB
:106580008B420CD3890192118B4208D3890192115D
:106590008B4204D389013AD0921100E08909C309E2
:1065A0008B4201D3CB01C01A524183098B4201D3E4
:1065B0008B01C01A524143098B4201D34B01C01ACF
:1065C000524103098B4201D30B01C01A5241C30847
:1065D0008B4201D3CB00C01A524183088B4201D3B6
:1065E0008B00C01A5241D9D243088B4201D34B00D1
:1065F000C01A5241411A00D20146634652415B1013
:10660000104601D34042002B00D5494270476346F3
:106610005B1000D3404201B5002000F005F802BD38
:106620000029F8D016E770477047C046D0400B1CD1
:106630001141203A03D49C46134118436346524209
:10664000934018437047C0468446101C62468C46EF
:10665000191C634600E0C0461FB500F08BFD002802
:1066600001D40021C8421FBD10B500F0DFFC40423C
:10667000013010BD10B500F07DFD002801DB0020C9
:1066800010BD012010BDC04610B500F073FD0028FC
:1066900001DD002010BD012010BDC04610B500F086
:1066A00005FD002801DC002010BD012010BDC04602
:1066B00010B500F0FBFC002801DA002010BD01201D
:1066C00010BDC046F0B54F464646C0B41604360C61
:1066D0009946330005042C0C070C150C63437E43CC
:1066E0006F4365431C0CAD1964199C46A64203D93F
:1066F00080235B02984647446346250CEF191D042E
:106700004B464A4343432D0C240464199918C91974
:1067100020000CBC90469946F0BDC046F0B55746E7
:106720004E4645464300E0B446028846760A1F0EB0
:10673000C40F002F47D0FF2F25D0002380259A4675
:106740009946F600ED042E437F3F434642465D02E4
:10675000D20F5B006D0A1B0E904640D0FF2B39D044
:1067600080220020ED00D20415437F3BFB184246F7
:106770005746591C62408C4607430F2F5CD86F491F
:10678000BF00C9598F46002E45D108239A46063BC3
:106790009946DAE7424602282DD0032800D1C3E00B
:1067A000012800D0A2E0002500260240D4B27602E3
:1067B000ED05760A2E43E407264330001CBC9046C4
:1067C0009946A246F0BD002E1AD104239A46033BF7
:1067D0009946BAE72A00511E8A41901CC6E701205B
:1067E000002DC3D0280001F0C9FB431F76309D4027
:1067F00043420020BAE70124FF2514400026D6E7D3
:10680000300001F0BBFB431F9E400023763047421F
:106810009A46994699E70C239A46093B994694E78C
:1068200080260024F603FF25C1E735004846B2E77D
:10683000350022004846AEE72904090C0800370C51
:106840003604360C2C0C7943704367437443060CB2
:1068500064183619B14203D9802149028846474459
:106860000004000C310409188D01681E8541890E51
:106870002943350CED19AD010D43290104D5012340
:1068800069081D4063460D4319007F31002925DD4D
:10689000680704D00F202840042800D004352801C0
:1068A00003D5274980330D401900FE29A3DC0124BC
:1068B000AD016E0A1440CDB279E78020C0030642D4
:1068C00007D0054205D128434602760A4446FF25F3
:1068D0006DE706437602760AFF2568E70124611A10
:1068E0001B2905DD14400025002660E76346CBE741
:1068F0002E002023CE40591A8D406B1E9D412E4301
:10690000730704D00F233340042B00D004367301E7
:1069100004D5012401251440002648E70124B601CE
:10692000760A1440002542E780260124F6032E4310
:106930007602760A1440FF2539E7C04618A3000006
:10694000FFFFFFF770B5002830D0C317C5185D40B2
:10695000C40F280001F012FB9E231B1A962B0DDC9E
:106960009622D21A95406A02520AD8B25202C00543
:10697000520AE40702432243100070BD992B19DC30
:106980009922D21A9540124A2A40690704D00F2151
:106990000D40042D00D00432510103D50C4B1A4098
:1069A0009F231B1A9201520AD8B2DFE7002400206D
:1069B0000022DBE705222E00121AB921D6402A0058
:1069C000C91A8A40551EAA4135001543DBE7C04667
:1069D000FFFFFFFBF8B556465F464D464446F0B410
:1069E0000F00FD0FAA4609037C002E005F00450F33
:1069F000490A7F0D2943C5001803BC46400A570FBA
:106A0000640DDB0F3843D2009A4500D1AAE06646F8
:106A1000A61B002E00DCFFE06346002B39D10300EB
:106A2000134300D0D9E06B0709D00F232B40042B70
:106A300005D02B1DAB42AD416D4249191D000B0223
:106A400000D482E0CA4B01349C4200D1FEE00A002F
:106A50005646C84BED081A405007640552020543DC
:106A6000120B640D002112030B0D1B056405120BA4
:106A70001A436308C04CF60714401C4364006408C2
:106A80003443280021003CBC90469946A246AB46C0
:106A9000F8BDB74B9C42C6D080231B041843382E48
:106AA00000DDEBE01F2E00DD1EE120239B1B9C463A
:106AB00003006746BB40984613004746F3403B43FC
:106AC0006746BA40571EBA4113430200F240EB1A20
:106AD0009D42B6411D008A1A7642911B0B0231D5A8
:106AE0004A02560A002E00D1B4E0300001F046FA06
:106AF0000300083B1F2B00DDB5E020222900D21A3D
:106B0000D1409E400A009D4032439C4200DDB1E0EE
:106B10001C1B631C1F2B00DDD5E020211400280066
:106B2000C91A8C40D8408D400443DA40681E854124
:106B300011002543002476E74146314300D134E279
:106B4000310045466B0700D06FE756464807ED0811
:106B5000C9080543864B9C4235D00A036405120BD5
:106B6000640D7FE76346E31A9B46002B00DC8BE055
:106B70006746002F3CD07E4FBC4200D153E78027B0
:106B80003F0438435B46382B00DCF7E00243501EDD
:106B900082410020D2B253194218AB4289411D00F4
:106BA000494289180B02CDD5714B01349C4200D16A
:106BB0003DE101206F4A6B080A4028401843D50781
:106BC000054351082FE72B000B4300D1CBE1802375
:106BD0001B030B431A03120B44E7013E002E6DD139
:106BE000AE1AB5429B41091A5B42C91A350075E7D6
:106BF0000700174300D116E701235B429C46E3449C
:106C00005B46002B00D0E0E0AA18AA429B4109187D
:106C10005B4259181500C5E7002E75D1661C760534
:106C2000760D012E00DCF3E0AE1AB0464545BF41BB
:106C30000E1A7F42F61B370200D48FE0551BAA4282
:106C4000B641411A76428E1B9A464BE756460022C1
:106C5000002507E7280001F091F920300300083BE8
:106C60001F2B00DC49E72A002838824000259C427F
:106C700000DC4DE73F49E41A1140D4E60243501EC0
:106C80008241D3B2002222E7002B00D0F3E0631C44
:106C90009C465B055B0D012B00DC9FE0344B9C4563
:106CA00000D1C3E0AA180918AA4280414042411805
:106CB000CD075208154349086446B4E62C4B9C4264
:106CC00000D0ECE6AFE611001F3CE1400C00202BA9
:106CD00000D17FE04021CB1A9A4015436A1E9541AE
:106CE0000021254300242DE733000700203BDF402F
:106CF0003B00202E70D04027BE1BB0400243501EE8
:106D0000824113430022E2E6002C4FD0184CA445E8
:106D100000D1ABE08024240476422143382E00DDEC
:106D2000DFE01F2E00DD43E12027BC1BA1460C0045
:106D30004F46BC40A0462C004746F4403C434F46DB
:106D4000BD406F1EBD41F1402C43151BAA4292412C
:106D5000411A5242891A64469A46BFE64146454660
:106D6000314300D0BEE6002600240025F2E6C046EE
:106D7000FF070000FFFF7FFFFFFF0F801F2B59DC85
:106D80002027FF1ABC46070063469F405B46B94672
:106D90001700DF40B8464F4643461F4363469A40BC
:106DA000531E9A415B463A43D840F4E60C002C430C
:106DB0005CD0F643002E55D1551BAA42A441411A7E
:106DC0006442091B9A46644688E6964FBC4200D04E
:106DD000D8E628E6002280E700208FE70B002B434F
:106DE000002C00D0C2E0002B00D101E103001343CE
:106DF00000D118E6AB18AB42B641091876427118BB
:106E00000A0200D409E1884A1D00114064460AE6DE
:106E1000002C5BD10E002E4300D08AE0010011430C
:106E200000D1C2E0010015009A46FCE5644600214D
:106E300000258FE620235B429C46DC446346070026
:106E4000DF405B46BC46202B00D1ACE040235F46D0
:106E5000DB1B98400243501E8241634613431A00D5
:106E6000002098E66F4CA44500D057E701001500BC
:106E700064469A46D7E5002C39D10C002C436ED0DD
:106E8000DB43002B1AD0674CA44568D0382B00DDBB
:106E9000A4E01F2B00DDAEE020240F00E41AA74081
:106EA000B9462F00DF40B846A3464F464446274325
:106EB0005C46A5406C1EA541D9403D43AD189542A6
:106EC0009B4109185B42591864466BE60C002C4341
:106ED00015D1010011437BD0010015009A46514C99
:106EE000A1E50D43691E8D410021ECB22DE74D4C0B
:106EF000A44534D0802424045B422143C6E7040027
:106F000014434ED0ED084C072C438025C9082D03AF
:106F1000294208D0C6082E4205D1D20841071143A4
:106F20000C009A463100620FC900E50011433D4C48
:106F300079E50600164300D175E5AE1AB046454521
:106F4000BF410E1A7F42F61B370200D4F4E5551BF1
:106F5000AA42B641411A7642891B9A4663E501006E
:106F6000150064465FE5002200257BE5002B3BD041
:106F70000300134315D0ED084B072B438025C908A8
:106F80002D03294207D0C4082C4204D141070B002D
:106F90002100D2081343C9005A0F1143DD00214CD0
:106FA00041E5204C3FE5002054E700260025D1E5CF
:106FB00034000F00203CE7403C00202E2BD040271F
:106FC000BE1BB1400D43691E8D4100212C43BCE620
:106FD000802100260903134C0025BBE50D43691EE3
:106FE0008D410021EDB269E7010015000D4C1AE555
:106FF0000100150017E51C000F00203CE7403C0095
:10700000202B0CD04027FB1A99400D43691E8D415F
:107010000021254352E70021D4E71D0092E500211D
:10702000F3E7C046FF070000FFFF7FFFF0B55F46B4
:1070300056464D464446F0B41F035C00DB0F9A46AB
:10704000194B0E034D00C90F8046360B6D0D8B4654
:1070500091463F0B640D9D4219D0134B9C421BD0AF
:107060000123A54206D018003CBC90469946A24692
:10707000AB46F0BDBE42F6D1C845F4D1D34510D0E1
:10708000002DF0D1304303005A1E9341EBE731004D
:1070900001230143E7D1E0E73A430123002AE2D18B
:1070A000DEE70023DFE7C046FF070000F0B55F46DC
:1070B000444656464D46F0B41F033C0B2C4F0E037E
:1070C0004D00A3465C008446360B6D0DC90F9046FB
:1070D000640DDB0FBD422BD0254FBC422ED0002DBE
:1070E0000ED130430700814678427841002C17D1F9
:1070F0005F463A4314D14B460020002B0AD006E0ED
:10710000002C02D15846024301D099421AD00123E3
:10711000484218433CBC90469946A246AB46F0BD57
:107120000028F2D058425841012240421043F1E772
:1071300037000743D0D002204042EBE75F461743B9
:10714000CDD0F8E7A542E2DC05DB5E45DFD808D00C
:1071500000205E45DED248424841012340421843A8
:10716000D8E7C445D3D80020C445F4D3D2E7C046FD
:10717000FF070000F0B55F464D4644465646F0B462
:107180001C03240BA4462F4C0F034D005E00C90FB7
:1071900080463F0B6D0D8B469146760DDB0FA54269
:1071A00020D0284CA64222D0002D12D13843444290
:1071B0004441002E20D0002C0DD05C4263410124BC
:1071C0005B421C4320003CBC90469946A246AB461D
:1071D000F0BD002E17D05B4519D05B465C42012301
:1071E0001C43EFE7390002240143EBD1D9E76146A4
:1071F00002241143E6D1D7E761460A43DBD10024DC
:107200000028DFD0E9E761460A43E4D1E5E7B5426B
:1072100003DD01225C421443D4E7B542CDDB674570
:10722000DBD809D000246745CCD259464C42614195
:10723000012449420C43C5E7C845CED80024C845BF
:10724000F3D3BFE7FF070000F0B55F4656464D4653
:107250004446F0B40D0399464E002B0B87B007004F
:10726000924680469B46760DCC0F002E69D06D4B22
:107270009E4235D05B468022DD001204430F13434B
:107280002B439B46C3009846674B00279C46002330
:10729000664401934A4615035000D20F53462D0B06
:1072A000400D914600D176E05E4A90426CD080223B
:1072B0005B0F120413435C4AED0094461D43534692
:1072C0000022DB00604449463618701C6140029081
:1072D00017430F2F00D9AFE05448BF00C759BF462E
:1072E0005B461F4300D088E000239B46984602334C
:1072F00008270193CEE74946022A6AD0032A00D123
:1073000009E2012A00D0BBE1114000220023002540
:107310009046CCB200212D030A0D12052D0B15430A
:10732000434A1B0515401D436D00E4076D082543C6
:107330004046290007B03CBC90469946A246AB4661
:10734000F0BD034352D05B46002B00D18AE1584682
:1073500000F014FE03000B3B1C2B00DD7BE11D2223
:10736000D31A3A0001005D46DA4008398D40130017
:107370008F402B439B46B8462E4B00279C4600234C
:1073800060444642019385E752462A432CD10025AA
:107390000023022297E752462A4321D0002D00D134
:1073A00054E1280000F0EAFD03000B3B1C2B00DD3C
:1073B00046E11D21CB1A51460200D9405346083AF6
:1073C000954093400D431B4A94466044404200223E
:1073D00079E7012400220C40124B0025904699E7E2
:1073E0000025002301226EE703226CE700239B4661
:1073F00098460133042701934CE703230C2701939C
:1074000048E700238025984600242D03054B81E79B
:107410005D464346019A6FE75D4643462100019A67
:107420006AE7C046FF07000001FCFFFF58A3000009
:10743000FFFF0F80F30300004246120C91461A0C26
:107440009446424617044A461B041B0C5A436046A6
:1074500090464A4642431000039262461C003F0C8D
:107460007A437C4342440192220C9246019A524450
:10747000904506D98246802040028046C24450464C
:107480000390100C049048462404240C1204121992
:1074900005922A0C2D042D0C68432C008246484688
:1074A0007C4350438146200C804657435744474411
:1074B000BA4503D9802040028046C144380C3F04BD
:1074C000B84648442404240C01900498A044404445
:1074D00004905846000C814658460404200C82460D
:1074E000070048465F434C4643436046604364465A
:1074F000834650464443380C8446E4186444A3420F
:1075000003D980235B029C46E34448463F04230C96
:107510003F0C2404E419574668436F4384464D46A4
:10752000504655434243380C814662444A445B44CA
:10753000944503D9802040028446654403983F0463
:10754000834604983F0C8446E344C345804140424F
:107550008246100484460198674484466744A344E5
:10756000BC46A345A4419946D44464428742BF41E6
:10757000D4458041E144A04699459B417F42404229
:10758000C8440743120CBA18A045A4415F423B000F
:1075900064422343D71843467D19DB0D6D021D431A
:1075A0005B465A02059B1A43531E9A415B46DB0D0C
:1075B0001A4343465B021343EA0107D501225C08E4
:1075C00013402343EA07029E13436D08574AB2183B
:1075D000002A4BDD580709D00F201840042805D099
:1075E000181D98429B415B42ED180300E80104D549
:1075F0004F4A15408022D200B2184E48824200DD28
:10760000E7E60124DB08680718436D02530580464E
:107610002D0B5B0D0C407DE6802259461203114272
:1076200008D0154206D115432D0398462D0B4C4624
:10763000414B6FE65D4615432D032D0B3E4B69E62E
:1076400003005546283B9D400023BCE6504600F011
:1076500095FC2030A8E60300283B9F400023BB4652
:10766000984689E600F08AFC203073E60124A61AC9
:10767000382E07DD00220C4000230025904649E605
:10768000029EA3E71F2E20DC20222C001800921B54
:10769000F040944093400443581E83411C43F540FE
:1076A000630709D00F232340042B05D023001C1DA2
:1076B0009C4292415242AD182B021FD50124002258
:1076C0000C4001230025904624E61F202C00404258
:1076D000821AD440202E1CD04022961BB5402B434A
:1076E000581E83410720234318400025002809D055
:1076F0000F2200251A401C00042AD8D12300680755
:107700006D022D0B0124DB08034398460C40002337
:1077100000E60025E3E780220124120315432D0330
:1077200098462D0B0C40044BF4E5C046FF030000C7
:10773000FFFFFFFEFE070000FF070000F0B5574601
:107740004E464546E0B40E001100F20F9246C500C9
:10775000420F180337037400400A4E0F7F0A30436C
:10776000CF4E17435A00640D520DDB0FC900B242D1
:1077700000D1E5E001267340A61AB446534500D176
:10778000AFE0002E00DC0DE1002A3AD103000B43EC
:1077900000D0E4E06B0709D00F232B40042B05D069
:1077A0002B1DAB42AD416D427F191D003B0200D441
:1077B00088E0BB4B01349C4200D110E13A00B94B48
:1077C00051461A4001235007ED0852026405054353
:1077D000120B640D0B400021280012030D0D120B3B
:1077E00064052D0515436208AF4CDB072C4014439C
:1077F000640064081C4321001CBC90469946A246C4
:10780000F0BDA74B9C42C5D080231B0418436346A0
:10781000382B00DDFDE01F2B00DD30E16246202328
:107820009B1A02009A40664690460A009940F24030
:1078300046464B1E99413243114363460200DA40EB
:10784000691A8D429B410D00BA1A5B42D71A3B025E
:1078500035D57A02530A98464346002B00D1C4E03E
:10786000404600F08BFB0300083B1F2B00DDC5E00A
:1078700020222900D21A4746D1409F400A009D404D
:107880003A439C4200DDC0E01C1B631C1F2B00DD43
:10789000E4E0202114002800C91AD8408C408D4013
:1078A0000443DA40681E854117002543002471E730
:1078B000424663461A4300D14CE2674645466B0791
:1078C00000D069E7012351467807ED08FA080B401C
:1078D000054373498C4238D012036405120B640DC2
:1078E00079E7002E00DC9AE0002A47D06C4A9442E7
:1078F00000D14FE78022120410436246382A00DC90
:1079000008E10143481E81410022C9B24919D21938
:10791000A942BF410D007F42BF183A0200D442E1A4
:107920005F4A0134944200D14EE101205D4A69086A
:107930003A4028400843D507054357089A4629E7A7
:1079400006000E4300D017E714E72900114300D1C9
:10795000F9E1802109030A431203120B3BE70123DB
:107960005B429846C4446346002B72D1691A8D422B
:107970009B413F1A5B42FF1A0D0068E702000A4371
:1079800000D107E7012252429046C4446246002AD1
:1079900000D0E6E06918A942B6413F187642F719CF
:1079A0000D00BAE7002E00D080E0621C5205520D97
:1079B000012A00DCF9E06A1A91464D45B6413A1AAF
:1079C0007642921B9046120200D499E04D1BA942C8
:1079D0008941C71B49427A1A90469A463CE752466B
:1079E0000123002513400022F5E6280000F0C6FA26
:1079F00020300300083B1F2B00DC39E72A00283821
:107A0000824000259C4200DC3EE7264FE41A1740E6
:107A1000C0E60143481E81410022C9B210E7002E92
:107A200000D0F1E0621C94465205520D012A00DCA0
:107A3000A0E01B4A944500D1C5E06918A9429241D3
:107A40003F185242D2194908D5070D4357086446DA
:107A5000A0E6134B9C4200D0D9E69BE611001F3CE8
:107A6000E1400C00202B00D180E04021CB1A9A404D
:107A700015436A1E95410027254300241FE76346EE
:107A80000200203BDA406346202B71D0402366463B
:107A90009B1B98400143481E814111430022CFE6C1
:107AA000FF070000FFFF7FFFFFFF0F80002C48D083
:107AB000CA4CA24200D1A2E07442A1468024240410
:107AC00027434C46382C00DDDBE01F2C00DD44E171
:107AD0004E462024A41B3E00A640A246B0464C467B
:107AE0002E00E640B4464646644626435446A5402A
:107AF0006C1EA54134002C434D46EF400D1B28E081
:107B00004A4643464D461A4300D0A5E600230024CA
:107B10000025DEE61F2A5ADC66462022921B06005C
:107B200096409146B04662460E00D6404246164305
:107B30004A4691404A1E9141020060463143C2408C
:107B4000E4E63C002C435AD0F443A146002C52D129
:107B50004D1BA9428941C71B49427F1A14009A460E
:107B600075E69E4A944200D0C7E613E600227FE7FE
:107B700000208FE7002C00D0C8E03B002B4300D151
:107B80000FE103000B4300D104E66918A9429B41B1
:107B90003F185B42DF193B0200D41AE1904B0D0005
:107BA0001F406446F6E59A4689E63A002A43002CCF
:107BB0005CD1002A75D102000A4300D1CAE0070057
:107BC0000D009A46E6E564460022002581E66246FD
:107BD0000600203AD6406246B046202A00D1B7E0DF
:107BE00040226646921B904001434246481E814116
:107BF000114300228AE6794CA24200D061E70700D7
:107C00000D0014009A46C5E5002C41D13C002C43E0
:107C100078D0F443A146002C20D0704CA24271D001
:107C20004C46382C00DDB2E01F2C00DDBCE02026E5
:107C3000341BA2463C005646B4404E46A0462C009B
:107C4000F440A446444666463443A4465446A54000
:107C500064466E1EB54125434C46E7406D188D4283
:107C600089413F184942CF19140056E6002A2FD106
:107C700002000A4300D184E007000D009A46574CE9
:107C800088E53D436F1EBD41ECB200270D1B60E748
:107C9000524CA24236D0744280263604A146374365
:107CA000BEE702000A4300D174E56A1A90464545D2
:107CB000B6413A1A7642921B9446120200D4F7E576
:107CC0004D1BA9428941C71B49427F1A9A4661E56B
:107CD00002000A433AD0ED087C072C438025FA08BD
:107CE0002D032A4208D0C7082F4205D145072C0092
:107CF0003A009A46C9080C43670FD200E5001743C3
:107D0000364C47E507000D00140043E53A002A43CE
:107D100043D002000A4319D0ED087C072C4380258C
:107D2000FA082D032A4207D0C6082E4204D147077D
:107D30003C003200C9080C43D700620FE50017432E
:107D40009A46264C26E50022002544E5234C21E5F1
:107D5000002049E700230025BBE54C463E00203CBF
:107D6000E6404C46B446202C31D040244E46A61B5B
:107D7000B7403D436C1EA54164462C4300270D1BB4
:107D8000E7E6802200231203144C0025A1E53D43C1
:107D90006F1EBD410027EDB260E707000D000F4CDC
:107DA000F8E407000D00F5E44E463C00203EF440A8
:107DB000A0464C46202C0ED040244E46A41BA74083
:107DC0003D436F1EBD4144460027254346E700273B
:107DD000CFE70D0073E50027F2E7C046FF0700007C
:107DE000FFFF7FFF0B0330B5134D1A0B4B005B0DEC
:107DF000C90F0024AB4211DD104CA34210DC8024DB
:107E0000640322430E4CE41A1F2C0CDD0D48C31AE8
:107E1000DA4013005C42002900D11C00200030BD74
:107E2000094BCC18FAE7E040084CA44663449A405A
:107E300013000343EEE7C046FE0300001D040000EC
:107E40003304000013040000FFFFFF7FEDFBFFFF82
:107E500070B5002830D0C317C4185C40C50F20008F
:107E600000F08CF8174B184A1B1AD21A1F2A18DD7B
:107E7000164AD21A9440002224035B05240B5B0DA2
:107E80000021100024030A0D1205240B1443104A8C
:107E90001B0514401C436400ED0764082C432100BB
:107EA00070BD210091400A000B21081AC4405B05F7
:107EB0002403240B5B0DE3E70025002300240022AC
:107EC000DEE7C0461E040000330400001304000077
:107ED000FFFF0F804200120E511C4302C9B270B561
:107EE0005D0AC40F012915DDE02189008C466D076C
:107EF0001B0B6244002128000D0D2D052B431C4D4A
:107F000052052B40520813435B00E4075B082343F0
:107F1000190070BD002A15D1002D1FD0280000F0D7
:107F20002DF80A281DDC0B232A001B1ADA40130047
:107F30000200153295400F4A1B03121A52051B0B03
:107F4000520DD7E7002D06D080221B0B12031343DE
:107F50006D07094ACEE7084A0023CBE70022002339
:107F6000C8E703000B3B9D402B000025E3E7C0461C
:107F7000FFFF0F8089030000FF0700001C21012381
:107F80001B04984201D3000C10391B0A984201D3FC
:107F9000000A08391B09984201D30009043902A2DA
:107FA000105C40187047C046040302020101010141
:107FB00000000000000000007FB51D000A4B060015
:107FC0001B68D868002A02D1084C230001E0130086
:107FD000074C0293009133002A000649019400F0F7
:107FE00021F800F023FEC04614020020AD990000E5
:107FF00098A30000A5A30000084B10B50400002BB7
:1080000002D0002100E000BF054B1868836A002BF6
:1080100000D09847200001F0F3FAC04600000000AD
:10802000D8A300000EB403B5010003AB044804CB91
:108030000068019300F016F902B008BC03B01847BD
:10804000140200200E4B70B500251E000D4CE41AE2
:10805000A410A54204D0AB00F35898470135F8E7C7
:1080600001F0D0FA084B00251E00084CE41AA410B9
:10807000A54204D0AB00F35898470135F8E770BD2E
:108080001C0200201C0200201C0200202C020020E8
:1080900010B5034B0100186800F066F810BDC0462B
:1080A0001402002010B5034B0100186800F016F808
:1080B00010BDC04614020020002310B59A4203D020
:1080C000CC5CC4540133F9E710BD0300821893421D
:1080D00002D019700133FAE77047000030B500296B
:1080E0003ED004390B68002B00DAC9181D4A13680A
:1080F0001400002B02D14B60116031E08B420DD98E
:108100000A688818834203D118685B6882180A607D
:108110004B60216024E08A4203D813005A68002A89
:10812000F9D11D685C198C420BD10968691858187F
:108130001960824214D110685268411819605A605F
:108140000EE08C4202D90C23036009E008680C1889
:10815000A24203D114685268201808604A6059602E
:1081600030BDC0465C110020032370B5CD1C9D437B
:10817000083506000C2D01D20C2505E0002D03DA90
:108180000C230020336040E0A942F9D81F4B1C6843
:108190001A002100002913D00B685B1B0DD40B2B98
:1081A00002D90B60CC181EE08C4202D163681360C8
:1081B0001AE04B6863600C0016E00C004968E9E7C0
:1081C000134C2368002B03D1300000F033FB2060F8
:1081D0002900300000F02EFB431CD1D00323C41C27
:1081E0009C43A0420AD12560200007220B30231DAA
:1081F0009043C31A09D05A42E25006E0211A3000D7
:1082000000F018FB431CEED1BAE770BD5C110020F2
:1082100058110020936810B5013B9360002B05DADC
:108220009469A34208DBCBB20A2B05D01368581C13
:1082300010601970C8B201E000F02CFC10BDF8B558
:1082400006000F001400D518AC4208D021783A007F
:108250003000FFF7DFFF0134431CF5D100E00020C0
:10826000F8BD0000F0B59FB006000F000292059324
:10827000002804D08369002B01D100F0D3FD7F4B8F
:108280009F4201D1776808E07D4B9F4201D1B768DA
:1082900003E07C4B9F4200D1F768BB891B070AD5DE
:1082A0003B69002B07D0002306AD6B6120336B7652
:1082B0001033AB763DE03900300000F043FC00287D
:1082C000F1D001204042D6E0059A111D12680591B7
:1082D000002A00DA7FE00992013423782E2B00D1A6
:1082E0008DE021780322684800F082FE002807D044
:1082F000654B2A68C01A4023834013432B60013426
:108300002178631C062261480293297600F070FEF2
:10831000002800D19DE05E4B002B00D090E00722AA
:10832000059B07339343083305936B69039A9B18A6
:108330006B61029C2378002B04D1029BE31A049307
:1083400012D003E0252BF8D00134F3E7049B029A06
:1083500039003000FFF773FF431C00D186E06A69E3
:10836000049B944663446B612378002B7ED00122EA
:10837000002352426A6002A95432521801342B6021
:10838000EB60AB601370AB6521780522414800F0CB
:108390002FFE002808D03F4B2A68C01A01238340D3
:1083A00013432B600134EFE72B68DA0604D5532220
:1083B000202102A8121811701A0704D553222B216C
:1083C00002A81218117022782A2A00D17CE7099B92
:1083D00000200A2105E05242EA60022213432B608A
:1083E0007AE72278303A092A04D84B4301349B18A3
:1083F0000120F6E7002800D16FE709936DE7637865
:108400002A2B0AD1059B02341A1D1B680592002BEA
:1084100001DA01235B42079363E700230A201A0075
:1084200001346B6021783039092904D84243013482
:1084300052180123F6E7002B00D152E7079250E7CC
:1084400005AB00933A00144B2900300000E000BF58
:1084500007E005AB00933A000F4B2900300000F015
:108460008BF80390039B013300D05EE7BB895B066A
:1084700000D526E70B981FB0F0BDC04610A5000040
:1084800030A5000050A50000E2A30000E6A3000014
:1084900000000000DCA300003F820000F7B51700D9
:1084A00001938A680B6900900C00934200DA130074
:1084B00022003B6043321278002A01D001333B6036
:1084C00023689B0602D53B6802333B600625236880
:1084D0001D401ED0230043331B785A1E934122684F
:1084E00092061CD53020E1184331087021005A1C37
:1084F00045310978A2184332023311700FE022008F
:108500000123193201990098089EB047431C0ED0F0
:108510000135E3683A689B1A9D42F0DBDAE72200F6
:10852000019943320098089DA847431C02D10120BD
:10853000404220E006232068E1683A6803400025B5
:10854000042B03D18D1AEB43DB171D40A36822696E
:10855000934201DD9B1AED180027BD420AD022008C
:1085600001231A3201990098089EB047431CDED0BF
:108570000137F2E70020FEBDF0B58BB006920A008D
:1085800043320793059004920A7E0C00109B6E2ADA
:1085900000D1ABE011D8632A22D009D8002A00D13B
:1085A000B5E0582A00D0C5E045310A70814A4FE055
:1085B000642A1DD0692A1BD0BCE0732A00D1AAE02E
:1085C00009D86F2A29D0702A00D0B3E02022096888
:1085D0000A43226037E0752A1FD0782A33D0A9E0F9
:1085E0000E001A684236111D196013683370A4E03A
:1085F00021681A68080606D4490604D5111D1960B9
:108600000023D55E02E0111D19601568002D3BDACC
:108610002D23049A6D42137036E021681A6808060B
:1086200006D4490604D51568111D1960ADB202E0E3
:10863000111D196015685F4B227E039308276F2A6E
:108640001DD00A271BE022007821453211705A4ABA
:1086500019680392081D226818600D68100602D47C
:10866000500600D5ADB2D30702D520231A432260AD
:108670001027002D03D1202322689A432260230073
:10868000002243331A7002E00A274A4B03936368BF
:10869000A360002B09DB0422216891432160002D97
:1086A00005D1049E002B11D07BE0002D79D0049ED3
:1086B00028003900FDF7CAFE039B013E5B5C2800E1
:1086C00033703900FDF73CFE051EF1D1082F09D1AA
:1086D0002368DB0706D563682269934202DC3023F6
:1086E000013E3370049B9B1B23612BE009681A68D1
:1086F000080607D4490605D5111D19601368A28A1A
:108700001A8004E0111D1960136862691A60002361
:10871000049E236116E01A68111D19601668002175
:108720006268300000F064FC002801D0801B6060AB
:10873000636803E026004236327001232361002380
:10874000049A1370079B09AA00932100069B0598C1
:10875000FFF7A4FE431C02D10120404227E0236919
:10876000320006990598079DA847431CF4D023685A
:1087700000259B070FD4099BE068984217DA180080
:1087800015E022000123193206990598079EB0478B
:10879000431CE1D00135E368099A9B1A9D42F0DB46
:1087A000E9E72600039B42361B7833708EE70BB057
:1087B000F0BDC046EDA30000FEA30000154B10B5B0
:1087C0001C68A36B002B15D11820FFF761FC124B1E
:1087D000A0630380114B01224380114B8380114B16
:1087E000C380114B0381052343810633838100231A
:1087F00002614361A46B0D4A206961690C4BFDF76E
:1088000061FF012200238018594120616161480005
:10881000400810BD140200200E330000CDABFFFF56
:10882000341200006DE6FFFFECDEFFFF2D7F954C5C
:108830002DF45158002370B5064C05000800236044
:1088400000F0C8FE431C03D12368002B00D02B602E
:1088500070BDC046502400200CB430B5164B9DB0FE
:108860000C1E1D6804DA8B2301202B6040421DE0A2
:10887000822302A99B008B810023029008619C4205
:1088800000D0631E8B604B6101235B42CB81209A39
:1088900021AB2800019300F053FC431C01DA8B2329
:1088A0002B60002C02D00023029A13701DB030BC44
:1088B00008BC02B01847C046140200200EB410B520
:1088C0009DB002A9029008610B488224886048612B
:1088D000012040421FABC881084804CBA4000068B7
:1088E00001938C8100F02CFC0023029A13701DB0C0
:1088F00010BC08BC03B01847FFFFFF7F1402002024
:1089000002780B78002A03D0013001319A42F7D067
:10891000D01A7047031C0A7801311A700133002AFB
:10892000F9D170470023C25C0133002AFBD1581EE5
:108930007047030030B5002A0DD00C7801335D1E5E
:10894000013A2C700131002CF5D19A189A4202D0CC
:108950001C700133FAE730BDF0B51E00454B87B0FF
:108960001B680192029308220B00059003911C786A
:1089700002995D1C09194878104001D02B00F6E7D8
:108980002D2C04D19D1C5C780123009304E0009001
:108990002B2C01D15C789D1C002E02D0102E0AD108
:1089A00062E0302C5ED120222B789343582B54D197
:1089B00010266C780235009F31007B1E9F412E4BA4
:1089C000FF183800FDF742FD380004913100FDF733
:1089D000B7FC00230322070094461800029A1219DC
:1089E00051780422114201D0303C07E06246114028
:1089F00017D03722012900D02032A41AA64210DD58
:108A00005A1C0BD0B84207D802D1049B9C4203DC0D
:108A100070430123201801E001235B422C780135CB
:108A2000DCE75A1C0BD10098059A431E9841124B63
:108A3000C01822231360019B002B0AD117E0009A73
:108A4000002A00D04042019A002A10D0039A002B3D
:108A500000D06A1E019B1A6009E03024002EAAD1C2
:108A60000826A8E70A26A6E7302C9CD0A3E707B083
:108A7000F0BDC04618020020FFFFFF7F10B51300B5
:108A80000A00010002480068FFF766FF10BDC046FB
:108A900014020020F8B505000F001400002804D0CF
:108AA0008369002B01D100F0BDF9234B9C4201D119
:108AB0006C6808E0214B9C4201D1AC6803E0204B7C
:108AC0009C4200D1EC68A369A360A3891B070AD567
:108AD0002369002B07D023682269FEB2981A6369C4
:108AE00098420FDB08E02100280000F02BF8002856
:108AF000F1D0012040421DE02100280000F024F9BF
:108B00000028F6D1A3680130013BA36023685A1CFA
:108B100022601F706369984205D0A3893000DB078B
:108B200008D50A2E06D12100280000F00DF90028F2
:108B3000DFD13000F8BDC04610A5000030A5000010
:108B400050A50000354B70B51D6806000C00002DC7
:108B500005D0AB69002B02D1280000F063F9304B3F
:108B60009C4201D16C6808E02E4B9C4201D1AC685C
:108B700003E02D4B9C4200D1EC68A3899AB2110707
:108B800023D4D10607D4092201203260373213439F
:108B9000A381404240E0530713D5616B002908D000
:108BA00023004433994202D03000FFF797FA0023A4
:108BB00063632422A3899343A38100236360236911
:108BC00023600822A3891343A3812369002B0BD1BF
:108BD000A023A2899B00134080229200934203D0DD
:108BE0002100300000F0B2F90123A289134005D022
:108BF0000023A36063695B42A36103E0910700D493
:108C00006369A36000202369834205D1130603D55D
:108C100040231A43A281013870BDC04614020020CF
:108C200010A5000030A5000050A5000010B50620DA
:108C300000F0AEFB012000F0E3FC0000F7B58A89EC
:108C400005000C0013075AD44B68002B02DC0B6C98
:108C5000002B19DDE76A002F16D000232E682B6049
:108C600080235B011A4001D0606D14E00123216A6A
:108C70002800B847431C0ED12B68002B0BD01D2BAE
:108C800001D0162B02D12E6000205AE04022A38989
:108C90001343A38155E0A3895B0706D56368C01A17
:108CA000636B002B01D0236CC01A00230200216AE1
:108CB0002800E76AB847A389421C06D129681D2904
:108CC0003AD8204ACA40D20736D5002262602269CB
:108CD0002260DB0405D5431C02D12B68002B00D198
:108CE0006065616B2E600029CED023004433994229
:108CF00002D02800FFF7F2F90020606321E00F693D
:108D0000002FC1D00B680F60DB1B0193002392077B
:108D100000D14B69A36003E0019B3F181B1A01932C
:108D2000019B002BB0DD019B3A00216A2800A66A56
:108D3000B0470028F0DCA389402201201343A3811F
:108D40004042FEBD010040200B6970B505000C00DB
:108D5000002B01D100201CE0002804D08369002BE7
:108D600001D100F05FF80B4B9C4201D16C6808E028
:108D7000094B9C4201D1AC6803E0084B9C4200D1F6
:108D8000EC680C22A35E002BE4D021002800FFF742
:108D900055FF70BD10A5000030A5000050A50000D3
:108DA00010B5024900F0B0F810BDC046498D000072
:108DB000002310B504000360436083608181436633
:108DC000C281036143618361190008225C30FFF7AF
:108DD0007CF9054B24626362044BA362044BE3629B
:108DE000044B236310BDC046D1930000F9930000EB
:108DF000319400005D94000070B568254B1E5D4302
:108E00000E0029007431FFF7AFF9041E08D00021CD
:108E10002A00016046600C30A0606832FFF755F907
:108E2000200070BD836913B50400002B28D1836432
:108E3000C3640365134B144A1B6882620193984212
:108E400001D101238361200000F020F86060200040
:108E500000F01CF8A060200000F018F80022E0608C
:108E600004216068FFF7A4FF01220921A068FFF731
:108E70009FFF02221221E068FFF79AFF0123A361FE
:108E800013BDC046D8A30000A18D0000F8B51D4B4E
:108E900006001D68AB69002B02D12800FFF7C2FF56
:108EA0004835AC686B68013B05D40C22A75E002FE7
:108EB00010D06834F7E72B68002B01D02D68F0E75D
:108EC00004213000FFF798FF28600028F6D10C231A
:108ED000336016E0012320005B42E3810233A3816B
:108EE00067662760A760676027616761A7615C307C
:108EF00008223900FFF7E9F820006763A763A76439
:108F0000E764F8BDD8A30000F7B504000700002609
:108F100001914834002C16D06368A5680093009B2B
:108F2000013B00930DD4AB89012B08D90E22AB5E17
:108F3000013304D029003800019B98470643683567
:108F4000EDE72468E6E73000FEBD0000F0B58B8950
:108F500091B006000C009B0726D40E23C95E0029A1
:108F600004DA8023A5891D4010D10CE001AA00F08D
:108F7000A1FA0028F5DBF023029D1B021D401A4BCD
:108F8000ED186B425D418027FF0001E0002540277E
:108F900039003000FFF7E8F800280CD1A3899A05C2
:108FA0001FD402221343A38123004733236023618C
:108FB0000123636115E080220C4BB362A38920601A
:108FC0001343A38120616761002D0AD00E23E15E67
:108FD000300000F081FA002803D00122A389134356
:108FE000A38111B0F0BDC04600E0FFFFA18D0000DD
:108FF000C9B28218904204D003788B4202D001306B
:10900000F8E70020704710B5884202D98B189842C3
:1090100001D3002305E09B1A013A08D3995C8154DF
:10902000FAE7934203D0CC5CC4540133F9E710BD96
:10903000F8B506000C001500002904D11100FFF757
:1090400093F8040018E0002A03D1FFF747F82C003A
:1090500012E000F067FA85420ED929003000FFF7D0
:1090600083F8071E07D021002A00FFF725F821000A
:109070003000FFF733F83C002000F8BDF0B58E68F3
:1090800085B007000C00039201939E4243D89023C1
:109090008A89DB001A423ED00325096923680198BA
:1090A0005B1A029363695D43EB0F5D19029B6D10C0
:1090B00001331B18AB4200D91D00530510D5290000
:1090C0003800FFF751F8061E14D0029A2169FEF706
:1090D000F3FFA289194B134080221343A38112E0AE
:1090E0002A003800FFF7A4FF061E0CD121693800C2
:1090F000FEF7F4FF0C23402201203B60A38940428D
:109100001343A38117E0029B2661F6182660656170
:10911000019EED1AA560019BB34200D21E003200F1
:1091200003992068FFF76FFF0020A3689B1BA360D3
:1091300023689E19266005B0F0BDC0467FFBFFFF87
:10914000F0B59FB0029005938B890F0016001B06A7
:1091500010D50B69002B0DD14021FFF705F83860C1
:109160003861002804D10C23029A01381360D8E03A
:1091700040237B61002306AD6B6120336B76103397
:10918000AB7634002378002B03D1A31B049312D0B9
:1091900003E0252BF9D00134F4E7A31B320039009A
:1091A0000298FFF76BFF431C00D1B4E06A69049B8F
:1091B000944663446B612378002B00D1ABE001221D
:1091C000002352426A6002A95432521801342B60C3
:1091D000EB60AB601370AB65534E21780522300015
:1091E000FFF706FF002807D00123801B83402A6871
:1091F000013413432B60EFE72B68DA0604D55322C2
:10920000202102A8121811701A0704D553222B210D
:1092100002A81218117022782A2A03D0099B002074
:109220000A210EE0059A111D12680591002A01DB42
:10923000099204E05242EA60022213432B60013497
:109240000BE02278303A092A04D84B4301349B18AA
:109250000120F6E7002800D0099323782E2B1ED199
:1092600063782A2B0AD1059B02341A1D1B680592CC
:10927000002B01DA01235B42079310E000230A2050
:109280001A0001346B6021783039092904D842432F
:10929000013452180123F6E7002B00D00792234E29
:1092A000217803223000FFF7A3FE002806D04023D8
:1092B000801B83402A68013413432B6021780622E7
:1092C0001B48661C2976FFF793FE002812D0194B25
:1092D000002B06D10722059B0733934308330593E0
:1092E00014E005AB00933A00134B2900029800E00C
:1092F00000BF07E005AB00933A000F4B290002982E
:10930000FFF73AF90390039B013304D06B69039A8A
:109310009B186B6135E7BB890B985B0601D5012073
:1093200040421FB0F0BDC046DCA30000E2A3000035
:10933000E6A30000000000007D90000070B504006E
:109340000D1E1F2D04D916230360012040421EE08C
:10935000426C002A04D08B00D2181368002B08D16D
:10936000200000F031F82A000100200000F01AF877
:109370000DE00020012B0AD0591C03D117332360C4
:10938000013004E00024280014609847200070BDDC
:1093900010B5034B01001868FFF7D0FF10BDC046A1
:1093A00014020020002370B5064C050008001100CF
:1093B000236000F0F7F8431C03D12368002B00D092
:1093C0002B6070BD5024002010B500F0DBF810BDFC
:1093D00070B50C000E25495F00F0B0F8002803DBE3
:1093E000636D1B18636503E0A289024B1340A381E0
:1093F00070BDC046FFEFFFFFF8B51F008B89050069
:109400000C001600DB0505D50E23C95E00220223E1
:1094100000F074F8A289054B28001340A3813200A4
:109420000E23E15E3B0000F01FF8F8BDFFEFFFFFE9
:1094300070B50C000E25495F00F060F8A389421C4E
:1094400003D1054A1340A38104E080225201134353
:10945000A381606570BDC046FFEFFFFF10B50E230E
:10946000C95E00F015F810BD70B5050008001100C8
:109470000022064C22601A0000F0BAF8431C03D107
:109480002368002B00D02B6070BDC0465024002004
:10949000002370B5064C05000800236000F062F858
:1094A000431C03D12368002B00D02B6070BDC04645
:1094B00050240020002370B5064C05000800110060
:1094C000236000F057F8431C03D12368002B00D021
:1094D0002B6070BD50240020002370B5064C0500A1
:1094E0000800236000F056F8431C03D12368002BCA
:1094F00000D02B6070BDC0465024002070B5050020
:10950000080011000022064C22601A0000F052F8F8
:10951000431C03D12368002B00D02B6070BDC046D4
:10952000502400200B1F1A68101F002A04DA891823
:1095300004390B68D01804387047000070B5050076
:10954000080011000022064C22601A0000F03AF8D0
:10955000431C03D12368002B00D02B6070BDC04694
:109560005024002058220120014B40421A607047CD
:109570005024002058220120014B40421A607047BD
:109580005024002058220120014B40421A607047AD
:10959000502400205822024B00201A607047C04619
:1095A0005024002058220120014B40421A6070478D
:1095B0005024002058220120014B40421A6070477D
:1095C0005024002058220120014B40421A6070476D
:1095D00050240020044A1368002B03D01818106090
:1095E00018007047014BF9E7601100205824002053
:1095F00058220120014B40421A607047502400203D
:10960000FEE7C046F8B5C046F8BC08BC9E467047A9
:10961000F8B5C046F8BC08BC9E4670478E060000F0
:10962000200600009E060000D4060000100700007F
:109630004A07000086070000AE070000EC070000A4
:10964000320800008E080000D2080000380900002F
:1096500084090000AC090000E6090000300A00009F
:10966000580A0000900A0000CA0A0000060B000019
:109670008C0B0000540C0000E40C0000420D0000B4
:10968000840D0000A60D0000AE0D0000900E00003D
:109690008E0600008E0600008E0600008E0600007A
:1096A000DC0E0000460F0000B00F0000FA0F0000B3
:1096B0005C100000E210000070110000BE110000FC
:1096C00008120000401200008C120000D8120000A6
:1096D0002413000072130000C813000008140000D7
:1096E00074140000A6140000F21400003E150000DF
:1096F0008A150000C6150000121600005E16000054
:109700008E0600008E0600008E060000C8160000BF
:10971000FA1600002C1700005817000094170000DC
:10972000C01700008E0600008E0600008E060000A6
:109730008E060000F21700003A1800008E060000A6
:109740008E06000086180000B4180000FE18000005
:109750008E0600008E0600008E0600002E19000006
:109760006019000092190000C4190000F0190000EF
:10977000281A0000541A00007E1A0000A81A0000DF
:10978000DA1A00000C1B00004C1B0000781B0000C4
:10979000AA1B0000D61B00008E0600008E060000EB
:1097A0008E0600008E0600008E060000081C0000D9
:1097B000341C0000601C00008C1C0000B81C000061
:1097C000F01C0000281D0000601D0000981D000016
:1097D000C41D0000F21D0000241E00008E060000C3
:1097E0008E0600008E0600008E0600008E06000029
:1097F0008E0600008E0600008E0600008E06000019
:109800008E0600008E0600008E0600008E06000008
:109810008E060000521E0000801E000066616C7300
:10982000650074727565006C697374206F6620251D
:1098300064206974656D73006F626A656374206F7C
:109840006620636C6173733A20256400537461630E
:109850006B20756E646572666C6F77000D0A564DED
:109860002050616E69633A2025730D0A00496E73BA
:10987000756666696369656E74206D656D6F727972
:1098800020666F72204D6963726F426C6F636B73F9
:10989000206F626A656374206865617000496E7349
:1098A000756666696369656E74206D656D6F727942
:1098B00020666F72204D6963726F426C6F636B73C9
:1098C00020737461636B00626164206F626A656318
:1098D0007420617420256C640A0025783A20256480
:1098E00020776F7264732C20636C6173734944201A
:1098F00025640A004865616465723A2025780A008B
:1099000009307825782C0A006D6973630073696EDD
:109910000025642025642025642025640A00426116
:1099200064207265636F726420666F756E64206474
:109930007572696E6720696E697469616C697A61B4
:1099400074696F6E210A004E6F7420656E6F7567C3
:109950006820726F6F6D206576656E206166746534
:109960007220636F6D70616374696F6E0A00526577
:1099700073746F72696E67202564207363726970F7
:1099800074732E2E2E0053746172746564002D2D35
:109990002D2D2D0A0050657273697374656E7420E5
:1099A0004D656D6F727920546573740A0A000A4917
:1099B0006E697469616C697A696E67204D656D6F57
:1099C00072790A004D656D6F727920696E746974E1
:1099D00069616C697A65643B2077726974696E6746
:1099E000207265636F7264732E2E2E0A00526563B7
:1099F0006F7264206174206F6666736574202564DD
:109A00003A2025642025642025642025642028250B
:109A10006420776F726473290A0046696E616C3A3C
:109A20002063757272656E74202564207573656499
:109A30002025642063302025642063312025640ABA
:109A4000006E6F6E6500726164696F0064697361B6
:109A5000626C65526164696F006D657373616765FF
:109A60005265636569766564007061636B65745205
:109A7000656365697665007061636B657453656ED7
:109A800064007265636569766564496E74656765CF
:109A9000720072656365697665644D6573736167AD
:109AA00065547970650072656365697665645374A1
:109AB00072696E670073656E64496E74656765727E
:109AC0000073656E64506169720073656E645374EF
:109AD00072696E67007365744368616E6E656C00D1
:109AE00073657447726F757000736574506F776536
:109AF00072007369676E616C537472656E67746827
:109B0000004E6F2066726565207461736B20656E10
:109B100074726965730057656C636F6D6520746F4F
:109B2000204D6963726F426C6F636B7321004D65EA
:109B30006D6F727920636C65617265642E00416C93
:109B40006C207461736B732073746F707065640044
:109B5000763035370020257320257300070000007C
:109B60000300000043616C6C696F7065006861738D
:109B7000546F6E6500706C6179546F6E650068613A
:109B800073536572766F00736574536572766F00F8
:109B900015000000010000000200000004000000A9
:109BA00005000000060000006E65740068617357D0
:109BB0006946690073746172745769466900737409
:109BC0006F70576946690077696669537461747587
:109BD00073006D79495041646472657373007468F1
:109BE000696E674465736372697074696F6E006350
:109BF0006C6561725468696E6744657363726970FD
:109C000074696F6E00617070656E64546F5468693A
:109C10006E674465736372697074696F6E0061701A
:109C200070656E64546F5468696E6750726F7065CA
:109C3000727479000D0E0F04050C0B0A0607080953
:109C40000D0E0F04050C0B0A0607080964697370F2
:109C50006C6179006C696768744C6576656C0000AE
:109C600000000000010000000200000003000000EE
:109C700004000000050000000600000007000000CE
:109C800008000000090000000A0000000B000000AE
:109C90000C0000000D0000000E0000000F0000008E
:109CA0001000000012000000140000001600000068
:109CB000180000001A0000001C0000001E00000038
:109CC0002000000023000000260000002900000002
:109CD0002C0000002F0000003200000036000000C1
:109CE0003A0000003E000000420000004600000074
:109CF0004B00000050000000550000005A0000001A
:109D000061000000680000006F00000076000000A5
:109D10007D000000840000008B0000009200000025
:109D200099000000A0000000A7000000AE000000A5
:109D3000B5000000BC000000C3000000CA00000025
:109D4000D1000000D8000000DF000000E6000000A5
:109D5000ED000000F4000000FB000000FF00000028
:109D6000000000000008080800080A4A4000000A35
:109D70005FEA5FEA0ED92ED36E19324489330C9212
:109D80004C924D0808000000048808080408048468
:109D90008488000A448A4000048EC48000000004C5
:109DA0008800000EC0000000000800012244881056
:109DB0000C9252524C048C84848E1C824C901E1E39
:109DC000C244924C06CA525FE21FF01EC13E0244DA
:109DD0008ED12E1FE24488100ED12ED12E0ED12E00
:109DE000C488000800080000048004880244880435
:109DF00082000EC00EC008048244880ED126C00422
:109E00000ED135B36C0C925ED2521C925C925C0EF9
:109E1000D010100E1C9252525C1ED01C901E1ED0F0
:109E20001C90100ED013712E12525ED2521C880854
:109E3000081C1FE242524C12549814921010101039
:109E40001E113B75B131113935B3710C9252524C20
:109E50001C925C90100C92524C861C925C92510E9B
:109E6000D00C825C1FE4848484125252524C113113
:109E7000312A44113135BB7112524C9252112A448D
:109E800084841EC488101E0EC808080E10080482A0
:109E9000410EC242424E048A400000000000001FF2
:109EA0000804800000000ED2524F10101C925C007B
:109EB0000ED0100E02424ED24E0C925C900E06C88E
:109EC0001C88080ED24EC24C10101C92520800087A
:109ED0000808024002424C1014981492080808081E
:109EE00006001B75B131001C925252000C92524C6C
:109EF000001C925C90000ED24EC2000ED0101000DA
:109F000006C8049808080EC807001252524F0011E4
:109F1000312A4400113135BB00124C8C9200112AB9
:109F20004498001EC4881E06C48C8486080808084D
:109F30000818080C881800000C836073656E736F36
:109F400072730074656D706572617475726500740A
:109F5000696C74580074696C74590074696C745A33
:109F600000746F756368526561640069326352659D
:109F700061640069326357726974650074667400C5
:109F8000656E61626C65446973706C6179007365BC
:109F900074506978656C006C696E650072656374F5
:109FA00000726F756E6465645265637400636972F4
:109FB000636C6500747269616E676C6500746578C6
:109FC0007400535049436C6173733A3A5350494398
:109FD0006C617373284E52465F5350495F547970D9
:109FE000652A2C2075696E74385F742C2075696E33
:109FF00074385F742C2075696E74385F7429007032
:10A000005F73706920213D204E554C4C002F5573D5
:10A010006572732F6A6F686E6D616C6F6E65792FF4
:10A020004C6962726172792F41726475696E6F3129
:10A03000352F7061636B616765732F73616E646543
:10A0400065706D69737472792F686172647761727B
:10A05000652F6E5246352F302E362E302F6C6962AA
:10A060007261726965732F5350492F5350492E63A3
:10A070007070000000000000000000003344000089
:10A08000F94300001F440000294400005944000027
:10A090001D4400000000000001000000020000005C
:10A0A000160000000400000005000000060000008B
:10A0B0000700000008000000090000000A0000007E
:10A0C0000B0000000C0000000D0000000E0000005E
:10A0D0000F0000001A0000001B0000001400000028
:10A0E0001300000011000000030000001000000039
:10A0F0001C0000001D0000001E00000012000000F7
:10A1000015000000170000001800000019000000F2
:10A11000FB21F93FFB2109407CD91240FB2119406A
:10A120007A6A1F407CD92240BBFD2540FB21294093
:10A130003A462C407A6A2F405C4731407CD9324005
:10A140009C6B3440BBFD3540DB8F3740FB213940F1
:10A150001BB43A403A463C405AD83D407A6A3F40A8
:10A160004C7E40405C4741406C1042407CD94240AC
:10A170008CA243409C6B4440AC344540BBFD454001
:10A18000CBC64640DB8F4740EB584840FB21494057
:10A1900083F9A200444E6E00FC291500D157270018
:10A1A000DD34F50062DBC0003C999500419043002E
:10A1B0006351FE00BBDEAB00B761C5003A6E240000
:10A1C000D24D42004906E00009EA2E001C92D1005F
:10A1D000EB1DFE0029B11C00E83EA700F53582000A
:10A1E00044BB2E009CE98400B4267000417E5F00D1
:10A1F000D6913900538339009CF439008B5F840079
:10A2000028F9BD00F81F3B00DEFF97000F980500FE
:10A21000112FEF000A5A8B006D1F6D00CF7E3600A4
:10A2200009CB2700464FB7009E663F002DEA5F002E
:10A23000BA277500E5EBC7003D7BF100F739070051
:10A2400092528A00FB6BEA001FB15F00085D8D002F
:10A25000300356007BFC4600F0AB6B0020BCCF0007
:10A2600036F49A00E3A91D005E619100081BE60028
:10A2700085996500A0145F008D40680080D8FF00BC
:10A2800027734D0006063100CA561500C9A8730091
:10A290007BE260006B8CC000020000000300000045
:10A2A000040000000600000000000040FB21F93F10
:10A2B000000000002D44743E000000809846F83CE9
:10A2C0000000006051CC783B00000080831BF03917
:10A2D0000000004020257A38000000802282E3360A
:10A2E000000000001DF369350000000000000000C0
:10A2F000315F0000515E0000A15F0000B55F00000B
:10A30000AB5F00002F5F0000235F0000C15F000013
:10A310004D5F00001F5F0000386800009667000076
:10A3200096670000946700002A6800002A68000011
:10A3300020680000946700002A6800002068000080
:10A340002A68000094670000306800003068000050
:10A3500030680000BA68000038740000F87200002D
:10A36000F8720000F6720000107400001074000013
:10A3700002740000F6720000107400000274000005
:10A3800010740000F67200001874000018740000C9
:10A3900018740000187600002C2066756E637469CE
:10A3A0006F6E3A2000617373657274696F6E20225C
:10A3B000257322206661696C65643A2066696C6564
:10A3C00020222573222C206C696E6520256425735C
:10A3D00025730A0043000000B4010020232D302B18
:10A3E0002000686C4C006566674546470030313296
:10A3F00033343536373839414243444546003031ED
:10A40000323334353637383961626364656600004B
:10A410002020202020202020202828282828202014
:10A42000202020202020202020202020202020202C
:10A4300088101010101010101010101010101010A4
:10A440000404040404040404040410101010101084
:10A45000104141414141410101010101010101015D
:10A460000101010101010101010101101010101091
:10A47000104242424242420202020202020202022E
:10A480000202020202020202020202101010102056
:10A4900000000000000000000000000000000000BC
:10A4A00000000000000000000000000000000000AC
:10A4B000000000000000000000000000000000009C
:10A4C000000000000000000000000000000000008C
:10A4D000000000000000000000000000000000007C
:10A4E000000000000000000000000000000000006C
:10A4F000000000000000000000000000000000005C
:10A50000000000000000000000000000000000004B
:10A51000000000000000000000000000000000003B
:10A52000000000000000000000000000000000002B
:10A53000000000000000000000000000000000001B
:10A54000000000000000000000000000000000000B
:10A5500000000000000000000000000000000000FB
:10A5600000000000000000000000000000000000EB
:04A5700000000000E7
:08A57400005CFF7F0100000004
:10A57C00FFFFFFFF0D990000B92000004C9A00006E
:10A58C0069270000599A00006D270000699A0000A5
:10A59C0071270000779A000075270000829A00004E
:10A5AC0031270000929A000045270000A69A00006F
:10A5BC0035270000B59A000079270000C19A0000E9
:10A5CC007D270000CA9A000081270000D59A000060
:10A5DC0085270000E09A000065270000E99A00003A
:10A5EC002D270000F29A00003D2700006D9B000013
:10A5FC0055330000759B0000513300007E9B00001A
:10A60C0059330000879B00005D330000AC9B0000B9
:10A61C001D360000B49B00004D360000BE9B0000B0
:10A62C0061360000C79B00006B360000D29B000017
:10A63C0057360000DE9B00002B360000EF9B00001D
:10A64C0041360000059C0000353600001E9C0000C1
:10A65C0021360000549C00008D36000018000000CC
:10A66C00439F00001D4100004F9F00003741000038
:10A67C00559F0000674100005B9F0000EB4000000D
:10A68C00619F0000A53E00006B9F000099410000F7
:10A69C00739F0000D13F0000809F00002542000006
:10A6AC008E9F000029420000979F00002D42000061
:10A6BC009C9F000031420000A19F00003542000029
:10A6CC00AD9F000039420000B49F00002142000001
:10A6DC00BD9F00001D4200000300000002000000AE
:10A6EC00080000000A000000FFFFFFFF0000000050
:10A6FC00010000000000020001000000FFFFFFFF4E
:10A70C000000000002000000000004000200000035
:10A71C00FFFFFFFF00000000030000000000080026
:10A72C00030000000000000010A5000030A5000090
:10A73C0050A5000000000000000000000000000018
:10A74C0000000000D4A30000000000000000000086
:10A75C0000000000000000000000000000000000ED
:10A76C0000000000000000000000000000000000DD
:10A77C0000000000000000000000000000000000CD
:10A78C0000000000B40100200FA4000039010000FB
:10A79C00C9430000E9460000256200000D010000DD
:04A7AC0000000000A9
:04000003000059E1BF
:00000001FF
